:020000040800F2
:1000000000000820CDAA0008C53D0008C73D000833
:10001000C93D0008CB3D0008CD3D000800000000B0
:10002000000000000000000000000000CF3D0008BC
:10003000D13D000800000000D33D0008D53D000878
:100040001DAB00081DAB00081DAB00081DAB000870
:100050001DAB00081DAB00081DAB00081DAB000860
:100060001DAB00081DAB00081DAB00081DAB000850
:100070001DAB00081DAB00081DAB00081DAB000840
:100080001DAB00081DAB0008DD3D00081DAB0008DE
:100090001DAB00081DAB00081DAB00081DAB000820
:1000A0001DAB0008F53D0008293E00081DAB000807
:1000B0005D3E00081DAB00081DAB00081DAB00082D
:1000C0001DAB00081DAB00081DAB00081DAB0008F0
:1000D0001DAB0008994100081DAB00081DAB0008CE
:1000E0001DAB00081DAB00081DAB00081DAB0008D0
:1000F000613E00081DAB00081DAB00081DAB0008E9
:100100001DAB00081DAB0008B13E00081DAB000888
:100110001DAB00081DAB0008B53E0008E93E000815
:100120001DAB00081DAB00081DAB00081DAB00088F
:100130001DAB00081DAB00081DAB00081DAB00087F
:100140001DAB00081DAB00081DAB00081DAB00086F
:100150001DAB00081DAB0008794200081DAB00086C
:100160001DAB00081DAB00081DAB00081DAB00084F
:100170001DAB00081DAB00081DAB0008000000000F
:100180001DAB00081DAB00081DAB00081DAB00082F
:100190001DAB00081DAB00081DAB00081DAB00081F
:1001A0001DAB00081DAB00081DAB00081DAB00080F
:1001B0001DAB00081DAB00081DAB00081DAB0008FF
:1001C0001DAB00081DAB0008000000001DAB0008BF
:1001D0001DAB00081DAB00081DAB00081DAB0008DF
:1001E0001DAB00081DAB00081DAB00081DAB0008CF
:0801F0001DAB00081DAB000867
:100200000348044B834202D0034B03B118477047A5
:100210005C0000205C000020000000000548064B48
:100220001B1AD90F01EBA301491002D0034B03B1F4
:10023000184770475C0000205C00002000000000B0
:1002400010B5064C237843B9FFF7DAFF044B13B11E
:100250000448AFF300800123237010BD5C00002030
:100260000000000020AB000808B5044B1BB1044996
:100270000448AFF30080BDE80840CFE7000000006D
:100280006000002020AB00080CB410B59CB01EAB81
:10029000029106916FF0004104910791084953F8CB
:1002A000042B0591002402A901931B9400F010F97E
:1002B000029B1C701CB0BDE8104002B0704700BF2C
:1002C0000802FFFF0EB430B59CB06FF000411FABC9
:1002D000049107910A4953F8042B029000240690D8
:1002E000084D0868019302A905951B9400F0F0F8E9
:1002F000029B1C701CB0BDE8304003B0704700BFCB
:10030000000000200802FFFF2DE9F0478F681D461E
:10031000AF420B680C46164636D8B1F90CC01CF437
:10032000906F0ED13D46184631462A4600F06EFBCE
:10033000A368DF1B2368A7602B4400202360BDE86F
:10034000F0874A69096902EB42025F1A02EBD27236
:100350006B1C52103B44934292BF914699461A46F9
:100360001CF4806F804611D0114600F071FA82466D
:1003700000B321693A4600F01BFCA38923F4906383
:1003800043F08003A38105E02F46CCE700F0BAFCE0
:10039000824658B10AEB0703A9EB0707A760C4F828
:1003A00010A0C4F8149023602F46BCE72169404692
:1003B00000F0CEFAA3890C2243F04003C8F80020D5
:1003C0004FF0FF30A381BAE72DE9F04F936817682B
:1003D00083B09246002B74D04FF0000B8B680A68F4
:1003E00081460C465D4645E0B4F90C3013F4906F3D
:1003F0002CD0D4E90401161A01EB410202EBD272AF
:10040000711C52102944914292BF904688460A4678
:100410005B0539D51146484600F01AFA01900028CC
:100420003DD03246216900F0C3FBA289019B22F432
:10043000906242F08002A2819819A8EB0606A6609D
:10044000C4F8148023612060A8462E4632465946DF
:1004500000F0DCFADAF80810A3682268A3EB0803BE
:100460003244491BA3602260CAF8081049B3D7E997
:1004700000B5083798461046002DF8D09D421E461C
:10048000B2D2A8462E46E1E70146484600F03AFCC3
:1004900003460028D0D12169484600F059FAA389C3
:1004A0000C2243F04003C9F800204FF0FF30A38135
:1004B00000220023CAF80820CAF8043003B0BDE8BF
:1004C000F08F00200023CAF8043003B0BDE8F08F9D
:1004D0002DE9F04F1C468B891D069DB0884681464C
:1004E000934603D50B69002B00F0F180002309939C
:1004F00043F22003ADF829309BF800307D4D039482
:100500000126002B73D0DA4603E01AF8013F002BD6
:1005100075D0252BF9D1BAEB0B0473D19AF80020D2
:10052000002A64D000234FF0FF32CDE905230AF101
:10053000010A049307938DF853301A9305E0049A47
:1005400006FA03F31A430492A2465446052214F80D
:10055000011B284600F0DCFAA346431B0028EED11D
:10056000049BD80644BF20228DF8532019079AF81F
:10057000001044BF2B228DF853202A2950D1039A12
:1005800011680432002903927CDB07919AF801106C
:100590002E295BD0584C0322204600F0B9FA38B11E
:1005A000049B001B4022824013430BF1010B049378
:1005B0001BF8011B51488DF82810062200F0A8FAFC
:1005C000002865D04E4B002B55D003AA00924D4B0E
:1005D000424604A94846AFF3008007467A1C06D07D
:1005E000099B3B4409939BF80030002B8BD1B8F852
:1005F0000C305B067AD409981DB0BDE8F08FBAEBD9
:100600000B04F4D023465A4641464846FFF77CFE89
:100610000130ECD0099B9AF80020234409937FE72E
:10062000A1F13002092A88BFD346B1D8079B00E068
:100630000134217803EB830302EB4303A1F1300281
:10064000092AF5D92E290793A346A3D19BF80110B7
:100650002A2927D1039B9BF802101A6805920433BC
:10066000002A0BF102000393B8BF4FF0FF3383461B
:10067000B8BF05938EE7039B073323F007030833C6
:100680000393ADE7494243F00203079104937DE7EA
:1006900003AA00921B4B424604A9484600F0F6FB11
:1006A00007469BE7A1F130020023092A05930BF1CD
:1006B000010B3FF66FAF1BF8011F03EB830302EB47
:1006C0004303A1F13002092AF5D9059362E74021DD
:1006D00000F0BEF8C8F80000C8F8100018B14023B8
:1006E000C8F8143002E70C23C9F800304FF0FF308F
:1006F00082E700BFACAC0008B4AC0008B8AC00089E
:10070000000000000903000870B50F4B0F4DAB420D
:10071000A3EB050607D0B610002455F8043B0134BE
:100720009847A642F9D80AF0FBF9094D094B5E1B20
:10073000AB424FEAA60606D0002455F8043B01342C
:100740009847A642F9D870BD9CAD00089CAD000842
:100750009CAD0008A0AD0008830730B547D0541EFB
:10076000002A3ED0CAB2034601E0013C39D303F867
:10077000012B9D07F9D1032C2CD9CDB205EB052512
:100780000F2C05EB054535D9A4F1100222F00F0C12
:1007900003F1100EE6444FEA121C1A46C2E9005556
:1007A000C2E9025510327245F8D10CF1010214F081
:1007B0000C0F03EB021204F00F0C13D0ACF1040386
:1007C00023F003030433134442F8045B9342FBD148
:1007D0000CF003042CB1C9B21C4403F8011BA34262
:1007E000FBD130BD64461346002CF4D1F9E7034633
:1007F0001446C0E71A46A446E0E700BF014B18685C
:10080000704700BF0000002070B5104E33680546E9
:100810000C46B3B12146284600F07EFC431C0CD0A8
:10082000C41C24F00304A04205D0211A284600F07D
:1008300073FC013001D0204670BD4FF0FF342046DC
:1008400070BD194600F068FC3060E3E778000020D6
:100850002DE9F843CD1C25F0030508350C2D38BFD4
:100860000C25002D064618DBA94216D8DFF8DC80DF
:1008700000F04EFCD8F80420A2B1144603E06368EF
:1008800022467BB11C4623685B1BF8D40B2B1FD878
:100890009442636854D053600CE00C233360002012
:1008A000BDE8F88329463046FFF7AEFF431C0446F7
:1008B00019D00560304600F02DFC04F10B00231D1B
:1008C00020F00700C21A1CBF1B1AA350BDE8F88312
:1008D00061199442256014BF5160C8F80410635137
:1008E00063684B60E6E7D8F804701FB33C467F6846
:1008F000002FFBD123683946304604EB030900F092
:100900000BFC814516D12368ED1A29463046FFF7C6
:100910007BFF01300ED02368D8F804202B442360DD
:10092000536883B1A34203D01A465B689C42FBD153
:100930000023B0E70C233360304600F0EBFBAEE75A
:10094000C8F80430B6E7C8F80470B3E778000020B0
:10095000002950D038B551F8043C0C1F002BB8BF0B
:10096000E418054600F0D4FB274A13682BB1A342D4
:100970000CD92168601883422CD06360284614602B
:10098000BDE8384000F0C6BBA3420FD81A465B68EA
:10099000002BF9D111685018844217D02CD3636012
:1009A00054602846BDE8384000F0B4BB11685018C8
:1009B000A04214D020D8216860188342EFD1186873
:1009C0005B680844C4E900035460EAE723680B4409
:1009D0001360E6E718685B6808442060CDE720688C
:1009E0000144501883421160DBD1D3E90004014473
:1009F000C2E90014D5E770470C232B602846BDE8F8
:100A0000384000F087BB00BF7C00002088420ED930
:100A10008B1883420BD900EB020C002A6ED0624681
:100A200013F801CD02F801CD9942F9D170470F2A90
:100A30000FD8034602F1FF3C002A5FD00CF1010CF5
:100A4000013B8C4411F8012B03F8012F6145F9D1CA
:100A5000704740EA01039B0751D1A2F1100370B522
:100A600001F1200C23F00F0501F1100E00F110042C
:100A7000AC441B095EF8105C44F8105C5EF80C5C3A
:100A800044F80C5C5EF8085C44F8085C5EF8045CB2
:100A900044F8045C0EF1100EE64504F11004E9D1AF
:100AA000013312F00C0F01EB031102F00F0400EB05
:100AB000031328D0043C24F003064FEA940C1E4490
:100AC0001C1F8E465EF8045B44F8045FB442F9D103
:100AD0000CF1010402F0030203EB840301EB840137
:100AE00002F1FF3C4AB10CF1010C013B8C4411F8BE
:100AF000012B03F8012F6145F9D170BD704702F158
:100B0000FF3C03469AE72246EAE700BF00000000E8
:100B100001F0FF01102A2BDB10F0070F08D010F8AE
:100B2000013B013A8B422DD010F0070F42B3F6D1B2
:100B3000F0B441EA012141EA014122F007047FF0CB
:100B400000070023F0E80256083C85EA010586EA22
:100B5000010685FA47F5A3FA87F586FA47F6A5FA5E
:100B600087F68EB9EED1F0BC01F0FF0102F007026A
:100B700032B110F8013B013A83EA010313B1F8D115
:100B80000020704701387047002D06BF35460338F6
:100B9000073815F0010F07D1013015F4807F02BF2F
:100BA000013015F4C03F0130F0BC0138704700BF80
:100BB000844641EA000313F003036DD1403A41D368
:100BC00051F8043B40F8043B51F8043B40F8043B27
:100BD00051F8043B40F8043B51F8043B40F8043B17
:100BE00051F8043B40F8043B51F8043B40F8043B07
:100BF00051F8043B40F8043B51F8043B40F8043BF7
:100C000051F8043B40F8043B51F8043B40F8043BE6
:100C100051F8043B40F8043B51F8043B40F8043BD6
:100C200051F8043B40F8043B51F8043B40F8043BC6
:100C300051F8043B40F8043B51F8043B40F8043BB6
:100C4000403ABDD2303211D351F8043B40F8043B56
:100C500051F8043B40F8043B51F8043B40F8043B96
:100C600051F8043B40F8043B103AEDD20C3205D366
:100C700051F8043B40F8043B043AF9D2043208D05E
:100C8000D2071CBF11F8013B00F8013B01D30B88D0
:100C900003806046704700BF082A13D38B078DD0AE
:100CA00010F003038AD0C3F10403D21ADB071CBF80
:100CB00011F8013B00F8013B80D331F8023B20F8EA
:100CC000023B7BE7043AD9D3013A11F8013B00F823
:100CD000013BF9D20B7803704B7843708B788370AB
:100CE00060467047024B01461868FFF7B1BD00BF70
:100CF00000000020024B01461868FFF729BE00BF24
:100D0000000000202DE9F041144641B30AB3064625
:100D10000D4600F013FA8442074602D8B4EB500F98
:100D200013D821463046FFF793FD804650B1BC42B0
:100D30002246294628BF3A46FFF73AFF2946304661
:100D4000FFF706FE4046BDE8F081A8464046BDE8F4
:100D5000F081A046FFF7FCFD4046BDE8F081BDE80C
:100D6000F0411146FFF774BD2DE9F84F92461F463A
:100D70000A698B68DDF828909A42B8BF1A46CAF80B
:100D8000002091F843300C46064613B10132CAF8F0
:100D90000020226891065FD5DAF800300233CAF8E5
:100DA0000030226812F0060F11461DD1E168994209
:100DB000D8BF114618DD4FF0000804F1190B05E00B
:100DC000E568DAF80030ED1A45450CDD01235A4696
:100DD00039463046C847013008F10108F0D14FF0DC
:100DE000FF30BDE8F88F216894F84330003B18BF0E
:100DF00001238A060AD5E1185A1C302081F84300E5
:100E0000224494F8451082F84310023304F143025F
:100E100039463046C8470130E1D02368DAF800503F
:100E2000216903F00603042BD4E902201BD08A4277
:100E300020DD4FF00008521A90441A34002501E0DA
:100E4000454517DA0123224639463046C847013066
:100E500005F10105F4D1C2E712F0060F0DD0003BF9
:100E600018BF0123D2E7401B8A4220EAE078E2DC87
:100E70000028E2DC0020BDE8F88FE168DAF80030F5
:100E80009942D8BF114696DCAEE700BF2DE9F04786
:100E9000174684B00A7E0C9D0C460646984601F122
:100EA000430C002A35D0A2F15803D9B2202969D8C1
:100EB000202B67D8DFE813F0E600660066006600C6
:100EC0006600660066006600660066006600AC00AC
:100ED00070006600660066006600700066006600CE
:100EE0006600660021008300C60066006600B6004A
:100EF0006600830066006600EC002B68226861696A
:100F0000181D286010061B6802D4520600F1E0800C
:100F100019600023E1462361CDF800803B4603AA17
:100F200021463046FFF720FF013020D023694A4692
:100F300039463046C047013019D02368E068DDF8F3
:100F40000C909B0718D5484516DD002504F1190AB9
:100F500004E0E068A0EB0903AB420DDD012352463B
:100F600039463046C047013005F10105F1D14FF057
:100F7000FF3004B0BDE8F0874845B8BF484604B02C
:100F8000BDE8F08784F84220012004F142090023E3
:100F9000206184F84330BFE72A682368111D1806D2
:100FA000296002D4590600F1958010680146002896
:100FB0006268C0F2938054484FF00A0E15E0206832
:100FC0002B6810F0800F53F8041B02D1400648BF75
:100FD00089B26F2A4C482B6014BF4FF00A0E4FF0B5
:100FE000080E0023626884F84330002AA26051DBB7
:100FF000236823F00403236000294BD1002A7BD10E
:10100000E146BEF1080F56D0ACEB0903236183E73C
:101010002B681A6804332B6004F1420984F84220DB
:101020000120B4E72B686268191D2960D3F800908D
:1010300000214846FFF76CFD002863D0A0EB0900B3
:101040006060A4E7236843F02003236078222F48E0
:1010500084F845202A6813F0800F52F8041B03D14E
:1010600013F0400F18BF89B22A60DA0744BF43F07B
:101070002003236019B9236823F0200323604FF075
:10108000100EAEE7582384F845301F482368E1E787
:101090002368DBE77546E146B1FBF5F305FB131A60
:1010A0000A46AA4210F80A1009F8011D1946F3D29F
:1010B000BEF1080FA8D12368DD07A5D562682369B2
:1010C0009A42A1DC302309F8013C09F1FF399BE782
:1010D00019801EE7B2F90010084668E72D20002AA3
:1010E000A26084F8430002DB23F0040323600A2596
:1010F00005484942AE46CEE7037884F8423004F111
:1011000042097EE7606842E7C0AC0008D4AC000842
:10111000704700BF704700BF38B5074D0022044636
:1011200008462A6009F0A4F9431C00D038BD2B689A
:10113000002BFBD0236038BDBC01002051F8043CDB
:10114000181F002BBCBF0B58C018704753B94AB9C1
:10115000002908BF00281CBF4FF0FF314FF0FF30BF
:1011600000F06AB9ADF1080C6DE904CE00F006F8A4
:10117000DDF804E0DDE9022304B070472DE9F04713
:10118000089D0E4604460F46002B4AD194468C45D6
:10119000B2FA82F260D942B1C2F12003974020FA3C
:1011A00003F30CFA02FC1F4394404FEA1C4E1FFA53
:1011B0008CF6B7FBFEF1230C0EFB117743EA0743D5
:1011C00001FB06F098420AD91CEB030301F1FF373B
:1011D00080F01581984240F21281023963441B1A53
:1011E000A4B2B3FBFEF00EFB103344EA034400FB51
:1011F00006F6A6420AD91CEB040400F1FF3380F086
:101200000081A64240F2FD806444023840EA014079
:10121000A41B00211DB1D4400023C5E90043BDE853
:10122000F0878B4205D90DB1C5E9000100210846C0
:10123000F5E7B3FA83F1002946D1B34202D38242E3
:1012400000F2F580841A66EB030201201746002D98
:10125000E5D0C5E90047E2E7002A40F09380A1EB22
:101260000C034FEA1C471FFA8CFE0121B3FBF7F673
:1012700007FB1630230C43EA00430EFB06F09842AE
:1012800008D91CEB030306F1FF3802D2984200F2A2
:10129000D08046461B1AA4B2B3FBF7F007FB10330D
:1012A00044EA03440EFB00FEA64508D91CEB0404E7
:1012B00000F1FF3302D2A64500F2B6801846A4EB37
:1012C0000E0440EA0640A5E7C1F120078B4022FA50
:1012D00007FC4CEA030C06FA01FE20FA07F426FA92
:1012E00007F344EA0E0400FA01F84FEA1C404FEA03
:1012F0001449B3FBF0FE1FFA8CF600FB1E3349EADB
:1013000003430EFB06F9994502FA01F20BD91CEBD7
:1013100003030EF1FF3A80F08580994540F2828008
:10132000AEF1020E6344A3EB0909A4B2B9FBF0F3DA
:1013300000FB139944EA094403FB06F6A64208D9C8
:101340001CEB040403F1FF3068D2A64266D9023BCD
:10135000644443EA0E40A41BA0FB02E6B442734679
:10136000B14652D34FD05DB1B8EB030264EB090430
:1013700004FA07F722FA01F31F43CC40C5E90074D1
:1013800000214CE7C2F1200120FA01F30CFA02FC23
:1013900026FA01F1964033434FEA1C471FFA8CFEB0
:1013A000B1FBF7F007FB1016190C41EA064100FBF0
:1013B0000EF68E4204FA02F408D91CEB010100F18A
:1013C000FF382DD28E422BD902386144891B9BB243
:1013D000B1FBF7F607FB161143EA014306FB0EF1DA
:1013E000994208D91CEB030306F1FF3814D2994245
:1013F00012D9023E63445B1A46EA004136E7394699
:10140000EDE6184602E7F045ADD2BEEB020366EB0F
:101410000C060138B146A6E74646ECE7034698E7D6
:101420004046D3E7D6467EE76444023847E708469D
:101430000DE7023E63442DE7704700BF00B500F0A2
:101440000700C0F1070CBCF1040F28BF4FF0040CDB
:10145000031D062B0FD9C31E4FF0FF3E0EFA0CF0F2
:1014600021EA000199400EFA03FE22EA0E0241EA47
:1014700002005DF804FB0023EEE70000064B074A7C
:101480001A6000225A609A60DA604FF400611961B4
:101490005A6114229A617047EC040020002C01402C
:1014A00000B583B00D4B1A6B42F480021A631B6BBC
:1014B00003F480030193019B094BD8680022114675
:1014C000C0F30220FFF7BAFF0001C0B2054B83F85A
:1014D000460340229A6003B05DF804FB00380240E6
:1014E00000ED00E000E100E082B0028802F00102BD
:1014F0001A700288C2F340025A700288C2F3800256
:101500009A700288C2F3C002DA700288C2F3001235
:101510001A710288C2F340125A710288C2F3801213
:101520009A710288C2F3C012DA710288C2F30022F3
:101530001A720288C2F340225A720288C2F38022D1
:101540009A720288C2F3C022DA720288C2F30032B1
:101550001A730288C2F340325A738278384B1A7079
:10156000828807EE902AF8EE677AC3ED017AC28886
:1015700007EE902AF8EE677AC3ED027A028907EE49
:10158000902AF8EE677AC3ED037A428907EE102AB3
:10159000B8EE477B9FED285B87EE056BFCEEC67BC4
:1015A000CDED017A9DF804201A75818907EE901A15
:1015B000F8EE677AC3ED067AC18907EE901AF8EE65
:1015C000677AC3ED077A018A07EE901AF8EE677A18
:1015D000C3ED087A418AD982818A07EE901AF8EE23
:1015E000677A9FED187A67EE877AC3ED0A7AC18A27
:1015F00007EE901AF8EE677A67EE877AC3ED097AFC
:10160000018B07EE901AF8EE677A67EE877AC3EDE2
:101610000C7A418B07EE901AF8EE677A67EE877ABC
:10162000C3ED0B7A084BA3FB0232D208074B1A60BA
:1016300002B07047AFF30080000000000000594086
:10164000C001002000008043CDCCCCCC080300209A
:1016500030B40B8804881B1BD1ED017A03F6B73C2C
:1016600041F26E74A44518D890ED027A06EE903AD5
:10167000F8EEE66A27EE267A284C2468284D2D6875
:10168000641B06EE904AF8EE666A27EE267A9FED16
:10169000256AC7EE066A77EEA67AD0ED016A9FED5D
:1016A000227AF4EEC77AF1EE10FA09DC9FED1F7A88
:1016B000F4EEC77AF1EE10FA04D5DFED1C7A01E002
:1016C000DFED197AC1ED017A07EE103AB8EEC77A6C
:1016D00027EE267ADFED166A37EE267AFDEEE77AF8
:1016E000F8EEE77A77EE877AFDEEE77A17EE900A62
:1016F000B0F57A7F06DB4DF6E053984204DD4DF6F7
:10170000E05001E042F26020022A02D080B230BCF8
:101710007047024B1A68024B1A60F7E71803002063
:10172000100300200000C8420000FA460000FAC67C
:101730000000004710B5092813D8DFE800F00513B2
:10174000212F3D4B5965717D414C01224FF4806141
:10175000204604F062FA00224FF48061204604F033
:101760005CFA10BD3A4C01224FF40061204604F0AF
:1017700054FA00224FF40061204604F04EFAF0E7DC
:10178000334C01224FF48051204604F046FA0022E7
:101790004FF48051204604F040FAE2E72C4C01223D
:1017A0004FF40051204604F038FA00224FF4005163
:1017B000204604F032FAD4E7254C01224FF4804150
:1017C000204604F02AFA00224FF48041204604F01B
:1017D00024FAC6E71E4C01224FF40041204604F0D3
:1017E0001CFA00224FF40041204604F016FAB8E734
:1017F000184C01221021204604F00FFA002210217B
:10180000204604F00AFAACE7124C012220212046BF
:1018100004F003FA00222021204604F0FEF9A0E79C
:101820000C4C01224021204604F0F7F9002240210F
:10183000204604F0F2F994E7064C0122802120466C
:1018400004F0EBF900228021204604F0E6F988E755
:10185000001802400004024038B5044600224FF44C
:101860008041814804F0D9F900224FF400717F488B
:1018700004F0D3F9002300E00133B3F5FA7FFBD382
:1018800001224FF48041784804F0C7F901224FF457
:101890000071764804F0C1F9002300E00133B3F58C
:1018A000FA7FFBD3631E032B39D8DFE803F0023A3B
:1018B0006FA66D4C01224FF40061204604F0ADF993
:1018C00000224FF48061204604F0A7F9002300E0D5
:1018D0000133B3F5FA7FFBD3654A136843F0400345
:1018E00013600023624A926812F0010F04D1B3F52D
:1018F0007A7F01D80133F5E75D490A6822F040029A
:101900000A6000E00133B3F5FA7FFBD301224FF404
:101910008061554804F081F9554BDD68ADB2284629
:1019200038BD524C01224FF48061204604F075F915
:1019300000224021204604F070F9002300E001332A
:10194000B3F5FA7FFBD34B4A136843F040031360AF
:101950000023484A926812F0010F04D1B3F57A7F50
:1019600001D80133F5E743490A6822F040020A60D2
:1019700000E00133B3F5FA7FFBD3012240213B485D
:1019800004F04BF93B4BDD68ADB2C8E7364C0122A1
:101990004FF48061204604F040F900224FF40061CA
:1019A000204604F03AF9002300E00133B3F5FA7F52
:1019B000FBD32F4A136843F04003136000232C4AE3
:1019C000926812F0010F04D1B3F57A7F01D8013388
:1019D000F5E727490A6822F040020A6000E0013377
:1019E000B3F5FA7FFBD301224FF400611E4804F0E7
:1019F00014F91F4BDD68ADB291E71C4C0122402168
:101A0000204604F00AF900224FF48061204604F0D9
:101A100004F9002300E00133B3F5FA7FFBD3154A44
:101A2000136843F0400313600023124A926812F0D7
:101A3000010F04D1B3F57A7F01D80133F5E70D49E1
:101A40000A6822F040020A6000E00133B3F5FA7F31
:101A5000FBD301224FF48061044804F0DEF8054B0B
:101A6000DD68ADB25BE700BF001002400014024029
:101A7000003401400050014008B5044805F072FFF1
:101A80000023034A1370034A136008BD08040020B2
:101A9000D60200200C0300202DE9F04F8FB0002467
:101AA00009940A940B940C940D94854B1A6B42F094
:101AB00020021A631A6B02F020020192019A1A6B3B
:101AC00042F080021A631A6B02F080020292029ABC
:101AD0001A6B42F004021A631A6B02F004020392BA
:101AE000039A1A6B42F001021A631A6B02F00102A8
:101AF0000492049A1A6B42F002021A631A6B02F003
:101B000002020592059A1A6B42F010021A631A6BD0
:101B100002F010020692069A1A6B42F008021A634B
:101B20001A6B02F008020792079A1A6B42F0400201
:101B30001A631B6B03F040030893089BDFF8908146
:101B400022464FF4C861404604F067F8DFF884B1DC
:101B500022463C21584604F060F85A4E22464B215A
:101B6000304604F05AF801221021304604F055F8AE
:101B7000554F22464FF44061384604F04EF801229A
:101B80004FF48041384604F048F8DFF84CA1224673
:101B900044F6F041504604F040F801224FF48051E1
:101BA000504604F03AF8DFF8349122464FF4C17100
:101BB000484604F032F822464FF47E41434804F090
:101BC0002CF8182309930A9401250B9509A940467E
:101BD00003F01AFF4FF4C86309930A950B940C9411
:101BE00009A9404603F010FF342309930A950B948A
:101BF0000C9409A9584603F007FF082309930A9596
:101C00000B9403230C9309A9584603F0FDFE5B23B4
:101C100009930A950B940C9409A9304603F0F4FE3D
:101C20004FF4F04309930A940B9409A9404603F03A
:101C3000EBFE4FF4406309930A950B940C9409A9A9
:101C4000384603F0E1FE4FF4804309930A950B9464
:101C500003230C9309A9384603F0D6FE45F6F0435A
:101C600009930A950B940C9409A9504603F0CCFEF5
:101C70004FF4C17309930A950B940C9409A9484633
:101C800003F0C2FE4FF4807309930A940B9409A9E0
:101C9000304603F0B9FE09950A940B9409A9484609
:101CA00003F0B2FE4FF47E4309930A950B940C9413
:101CB00009A9064803F0A8FE0FB0BDE8F08F00BFE9
:101CC00000380240000002400010024000180240AC
:101CD000001402400008024000040240000C0240D0
:101CE0002DE9F04192B02822002108A8FEF734FD2A
:101CF00000240294039404940594069407942A4BB8
:101D00005A6C42F400525A645A6C02F40052019226
:101D1000019A1A6B42F010021A631B6B03F0100356
:101D20000093009B4FF480530293022503954FF0DC
:101D30000308CDF81080052707971C4E02A93046EE
:101D400004F0D7FA4FF4005302930395CDF81080B6
:101D500005940694079702A9304604F0CAFA4FF496
:101D6000806308934FF4827309934FF470630A936E
:101D70000B950C944FF400730D9318230E930F944E
:101D80001094072311930A4C08A9204605F02EFC55
:101D9000636823F010036360636823F008036360E3
:101DA00012B0BDE8F08100BF0038024000100240D0
:101DB000003401402DE9F04192B02822002108A80A
:101DC000FEF7CAFC0024029403940494059406943C
:101DD0000794294B1A6C42F480421A641A6C02F47C
:101DE00080420192019A1A6B42F002021A631B6B45
:101DF00003F002030093009B4FF40053029302256B
:101E000003954FF00308CDF81080052707971B4E68
:101E100002A9304604F06DFA4FF400430293039593
:101E2000CDF8108005940694079702A9304604F077
:101E300060FA08944FF4827309934FF470630A9325
:101E40000B9501230C934FF400730D9310230E9305
:101E50000F94109407231193094C08A9204605F00C
:101E6000C5FB636823F010036360636823F0080315
:101E7000636012B0BDE8F081003802400004024007
:101E8000003800402DE9F04192B02822002108A836
:101E9000FEF762FC002402940394049405940694D3
:101EA0000794294B5A6C42F480125A645A6C02F41B
:101EB00080120192019A1A6B42F020021A631B6B86
:101EC00003F020030093009B8023029302250395D7
:101ED0004FF00308CDF81080052707971B4E02A985
:101EE000304604F006FA4FF4807302930395CDF860
:101EF000108005940694079702A9304604F0F9F97A
:101F00004FF4806308934FF4827309934FF4706326
:101F10000A930B950C944FF400730D9318230E93B2
:101F20000F94109407231193094C08A9204605F03B
:101F30005DFB636823F010036360636823F00803AC
:101F4000636012B0BDE8F081003802400014024026
:101F5000005001402DE9F04192B02822002108A84C
:101F6000FEF7FAFB0024029403940494059406946B
:101F70000794294B5A6C42F400125A645A6C02F4CA
:101F800000120192019A1A6B42F001021A631B6B54
:101F900003F001030093009B202302930225039585
:101FA0004FF00308CDF81080082707971B4E0DEB64
:101FB0000701304604F09DF9802302930395CDF884
:101FC00010800594069407970DEB0701304604F046
:101FD00090F908944FF4827309934FF470630A9355
:101FE0000B9501230C934FF400730D9318230E935C
:101FF0000F94109407231193094C08A9204605F06B
:10200000F5FA636823F010036360636823F0080344
:10201000636012B0BDE8F081003802400000024069
:102020000054014010B586B000240194029403943A
:10203000049405941D4B1A6C42F001021A641B6C47
:1020400003F001030093009B194BD86822462146F8
:10205000C0F30220FFF7F2F90001C0B2154B83F87C
:102060001C034FF080521A604FF47A73ADF80430BD
:102070000294114B0393049401A94FF0804006F0A1
:1020800005F94FF080431A6822F080021A609968BF
:102090000A4A0A409A605A6822F070025A609A68A6
:1020A00022F080029A6006B010BD00BF00380240E6
:1020B00000ED00E000E100E040D10C00F8BFFEFFC1
:1020C00010B586B0002401940294039404940594FE
:1020D0001C4B1A6C42F008021A641B6C03F00803D4
:1020E0000093009B184BD86822462146C0F302207B
:1020F000FFF7A4F90001C0B2144B83F832034FF488
:1021000080225A6042F21073ADF8043002944FF40A
:102110000C73039304940E4C01A9204606F0B6F804
:10212000236823F080032360A2680A4B1340A36056
:10213000636823F070036360A36823F08003A360E7
:1021400006B010BD0038024000ED00E000E100E004
:10215000000C0040F8BFFEFF10B586B000240194CB
:1021600002940394049405941A4B1A6C42F02002D2
:102170001A641B6C03F020030093009B164BD86875
:1021800022462146C0F30220FFF758F90001C0B2F1
:10219000124B83F837034FF400025A6040F2973332
:1021A000ADF804300294632303930D4C01A920463B
:1021B00006F06CF8236823F080032360636823F043
:1021C000700343F010036360A36823F08003A360EF
:1021D00006B010BD0038024000ED00E000E100E074
:1021E0000014004010B586B00024019402940394BA
:1021F000049405941A4B1A6C42F010021A641B6C7A
:1022000003F010030093009B164BD868224621462A
:10221000C0F30220FFF712F90001C0B2124B83F89D
:1022200036034FF480025A604BF2AF33ADF80430FE
:102230000294132303930D4C01A9204606F026F8BF
:10224000236823F080032360636823F0700343F066
:1022500010036360A36823F08003A36006B010BD81
:102260000038024000ED00E000E100E00010004016
:102270002DE9F04100239E4A13609E4A13609E4A56
:1022800013609E4A13609E4A13609E4A13709E4AD2
:1022900013809E4A13609E4A13609E4A13709E4AA2
:1022A000137005E09D4A002122F8131001339BB200
:1022B0000E2BF7D9994B41F211121A80984B00223C
:1022C000DA81DA701A711A821A735A735A719A7112
:1022D000DA72DA711A725A729A725A709A701A70A5
:1022E000904D2A80904C228000226A606260AA6031
:1022F000A2608E4E9C46BCE80F000FC6DCF8003092
:1023000033808B4E95E80F0086E80F00894D94E8E6
:102310000F0085E80F00884BDA6842F00102DA60AE
:102320001A6842F001021A6003F58063DA6842F02D
:102330000102DA601A6842F001021A6003F51433F0
:10234000D3F8B82022F00102C3F8B8204FF00062A1
:10235000DA604FF00072DA60784A02F1080353E85D
:10236000003F43F08003083242E800310029F3D1F6
:10237000734BD3F8B82042F01002C3F8B820D3F85A
:10238000B82042F00402C3F8B8204FF00062DA60CF
:102390004FF00072DA606B4AD3F8B83003F0C00334
:1023A000402B7BD0664BC3F8C020674AC3F8C420DB
:1023B0000024664B1C60664B1C60664F2246082159
:1023C000384603F02AFC22460421384603F025FC57
:1023D000DFF8A48122464FF48071404603F01DFCD3
:1023E00022461021384603F018FC5B4E22464FF47B
:1023F0008061304603F011FC584D224608212846E2
:1024000003F00BFC22460121284603F006FC22467D
:102410000221284603F001FC22464FF400613046B9
:1024200003F0FBFB22462021384603F0F6FB07F5BC
:10243000006701224FF48061384603F0EEFB484C00
:1024400001224021204603F0E8FB01224FF48041A5
:10245000384603F0E2FB01224FF48041204603F0AE
:10246000DCFB01224FF48041304603F0D6FB012211
:102470004021284603F0D1FB01224FF48051304621
:1024800003F0CBFB01221021284603F0C6FB0121FB
:10249000404603F0BBFB40B1BDE8F081284BC3F8D8
:1024A000C420294AC3F8C02082E74FF4807128462F
:1024B00003F0ACFB0028EFD12A4806F00FF82A4BB6
:1024C000186018B1294B01221A70E5E71E231A463D
:1024D0002749284806F052F8234C2060214806F08E
:1024E0000FF820600023084A1380064A1370E9E7BA
:1024F0003003002018030020140300202C030020C8
:1025000024030020D9020020D402002084020020ED
:1025100080020020D8020020D7020020B002002054
:102520001802002050020020400200202C0200204F
:1025300070020020600200200010004000100140E6
:1025400000640240DC02002028100140200300202B
:102550001C0300200008024000040240000002406A
:102560000014024038AB000888020020000300205D
:10257000900200203CAB0008000C024010B5002483
:1025800005282CD8DFE800F0030812171C26154890
:1025900002F038F9204610BD124C6421204602F0AA
:1025A000EBF9204602F049FA80B2F4E70D4802F058
:1025B000C3F92046EFE70C4802F024F92046EAE789
:1025C000094C6421204602F0D7F9204602F035FA82
:1025D00080B2E0E7044802F0AFF92046DBE720468E
:1025E000D9E700BFB80500207005002038B50C46BB
:1025F0000138032823D8DFE800F0023B5B7C00228F
:102600004FF480414B4803F008FB00224A4B9B6883
:1026100013F0020F04D1B2F5FA7F01D80132F5E7C9
:10262000454B9C810022444B9B6813F0010F04D161
:10263000B2F5FA7F01D80132F5E73F4BDB683D4D3B
:1026400001224FF48041284603F0E7FA3B4C012277
:102650004021204603F0E1FA01224FF48051284640
:1026600003F0DBFA01221021204603F0D6FA38BD30
:1026700000224021314803F0D0FA0022304B9B6801
:1026800013F0020F04D1B2F5FA7F01D80132F5E759
:102690002B4B9C8100222A4B9B6813F0010F04D125
:1026A000B2F5FA7F01D80132F5E7254BDB68C6E7C2
:1026B00000224FF480511F4803F0AFFA00221E4B56
:1026C0009B6813F0020F04D1B2F5FA7F01D80132F2
:1026D000F5E7194B9C810022174B9B6813F0010F03
:1026E00004D1B2F5FA7F01D80132F5E7124BDB686D
:1026F000A5E700221021114803F08FFA0022104BA9
:102700009B6813F0020F04D1B2F5FA7F01D80132B1
:10271000F5E70B4B9C810022094B9B6813F0010FDE
:1027200004D1B2F5FA7F01D80132F5E7044BDB683A
:1027300085E700BF0004024000380040000002406E
:10274000005401402DE9F84305460F4616461C4645
:10275000AF4B00221A600121AE4803F057FA00285F
:1027600000F0D2802B8803F0010323702B88C3F381
:10277000400363702B88C3F38003A3702B88C3F3DB
:10278000C003E3702B88C3F3001323712B88C3F3BA
:10279000401363712B88C3F38013A3712B88C3F399
:1027A000C013E3712B88C3F3002323722B88C3F378
:1027B000402363722B88C3F38023A3722B88C3F357
:1027C000C023E3722B88C3F3003323732B88C3F336
:1027D000403363736B883B80AB8833806B89E381C4
:1027E000AB8907EE903AF8EE677A9FED8B7A67EE49
:1027F000877AC7ED017AEB8907EE903AF8EE677AAF
:1028000067EE877AC7ED027A2B8A07EE903AF8EEE8
:10281000677A67EE877AC6ED017A6B8A07EE903A9F
:10282000F8EE677A67EE877AC6ED027AAA8A7B4B62
:102830005A83EB8ABB812B8BB3816378002B00F02A
:10284000958001220821764803F0E7F9A378002B50
:1028500000F0928001220421714803F0DEF9E37850
:10286000002B00F08F8001224FF48071694803F043
:10287000D4F92379002B00F08C80012210216848C4
:1028800003F0CBF96379002B00F0898001224FF42B
:102890008061644803F0C1F9A379002B00F08680C1
:1028A00001220821604803F0B8F9637A1BB1E3798B
:1028B000002B40F08180002201215B4803F0ADF93C
:1028C00000224FF40061574803F0A7F9A37A1BB127
:1028D000237A002B40F0868000220221524803F028
:1028E0009CF9002220214E4803F097F9237B1BB965
:1028F0004E4B7B604E4BBB60637B1BB94B4B736095
:102900004B4BB360BDE8F8834FF48071464803F049
:102910007DF901287FF426AF464805F0DFFD3C4BEA
:10292000186000287FF41EAFDFF80C91484605F0D0
:10293000EBFEDFF8DC80C8F80000484605F0C2FE78
:10294000C8F800001E222946484605F0E9FDC8F8EF
:1029500000001E222946484605F018FFC8F800006E
:10296000344805F0CDFDC8F80000FBE60022082140
:102970002B4803F052F969E700220421284803F0AC
:102980004CF96CE700224FF48071224803F045F9BE
:102990006FE700221021224803F03FF972E700227E
:1029A0004FF480611F4803F038F975E700220821D1
:1029B0001D4803F032F978E747F6FF710320FFF76F
:1029C00015FE47F6FF710320FFF710FE01224FF4BA
:1029D0000061144803F021F901221146124803F066
:1029E0001CF973E747F6FF710420FFF7FFFD47F678
:1029F000FF710420FFF7FAFD01222021084803F0AF
:102A00000CF901220221084803F007F96EE700BF24
:102A100088020020000C02400000803BB002002031
:102A20000008024000040240000002400000204173
:102A30000AD7233C38AB00083CAB0008844600882A
:102A4000012304E03CF81320504001331BB28B42B9
:102A5000F8DB704710B50E4B1B8841F21112934200
:102A600005D047F2777293420FD10E2400E00D2477
:102A70002146FFF7E3FF074B1880074B33F814306C
:102A8000984214BF0020012010BD0020FCE700BFC9
:102A9000D2020020D00200209002002010B504468F
:102AA00001210A4803F0B2F808B1012010BD08481E
:102AB00005F014FD08B10120F8E71E222146054863
:102AC00005F064FE024805F01BFDEFE7000C024034
:102AD00038AB000848AB000838B5044601210D4862
:102AE00003F094F808B1012038BD0B4805F0F6FC5E
:102AF00008B10120F8E7094D2B681E22214608483D
:102B000005F03CFD2B681E332B60034805F0F8FCF4
:102B1000EAE700BF000C024038AB00088402002046
:102B200048AB000810B501210B4803F06FF808B15D
:102B3000012010BD094805F0D1FC08B10120F8E7DB
:102B4000074C204605F0E0FD204605F0BBFD03489C
:102B500005F0D6FCEDE700BF000C024038AB0008E2
:102B600048AB00088C4600220CE033B9074BDB6908
:102B700013F08003F9D00123F7E7815C034B9962DE
:102B8000013292B26245F1D3704700BF001001409C
:102B90000D4B1B78002BFBD10C4BD3F8B82022F047
:102BA0000102C3F8B820D3F8BC206FF30F02104322
:102BB000C3F8BC00D3F8B82042F00102C3F8B82033
:102BC000014B01221A707047D802002000640240B5
:102BD00072B6FEE700B585B000230093019302931F
:102BE00003932B482B4A02604FF4403242608360CB
:102BF00001220261836180F82030C362264981622C
:102C0000C3600521C16180F83030426101F0CEFD22
:102C1000002831D109230093012301930723029354
:102C200069461B4801F0AAFF40BB0823009302231A
:102C300001936946164801F0A1FF08BB02230093E7
:102C4000032301936946124801F098FFD0B90A2383
:102C500000930423019369460D4801F08FFF98B952
:102C60000B230093052301936946094801F086FF71
:102C700060B905B05DF804FBFFF7AAFFFFF7A8FFF6
:102C8000FFF7A6FFFFF7A4FFFFF7A2FFFFF7A0FFE4
:102C9000B8050020002001400100000F00B585B0FC
:102CA000002300930193029303931448144A026093
:102CB0004FF44032426083600361836180F82030CA
:102CC000C362104A8262C3600122C26180F8303060
:102CD000426101F06BFD68B90F230093012301935A
:102CE000072302936946054801F048FF20B905B063
:102CF0005DF804FBFFF76CFFFFF76AFF700500202B
:102D0000002201400100000F2DE9F041B4B0002184
:102D10002D912E912F9130913191329133912791B4
:102D2000289129912A912B912C91902203A8FDF7AB
:102D300013FD4023039303A802F066FB002840F034
:102D40009E80504B5A6C42F010025A645A6C02F04A
:102D500010020292029A1A6B42F001021A631B6B74
:102D600003F001030193019B4FF4007327934FF08D
:102D70000208CDF8A0800327299700242A942B94D9
:102D800007262C96404D27A9284603F0B2FA4FF4A7
:102D900080632793CDF8A08029972A942B942C96B2
:102DA00027A9284603F0A5FA384BD3F8B82022F01B
:102DB000F05242F00062C3F8B820D3F8B82022F0F5
:102DC000C00242F04002C3F8B820D3F8B82042F461
:102DD0004032C3F8B820D3F8B82022F49072C3F878
:102DE000B820D3F8B82022F40072C3F8B820D3F882
:102DF000B82042F48062C3F8B820D3F8B82022F497
:102E0000C052C3F8B820D3F8B82022F4C042C3F8A7
:102E1000B820D3F8CC2022F00402C3F8CC201C4BFD
:102E2000D86822462146C0F30220FEF707FB0001C6
:102E3000C0B2184B83F8250320225A604FF4E133C7
:102E40002D932E942F9430940C23319332943394F9
:102E500004F1804404F588342DA9204605F0B6FA23
:102E6000636823F490436360A36823F02A03A3609C
:102E7000236843F00103236034B0BDE8F081FFF71D
:102E8000A7FE00BF0038024000000240006402407C
:102E900000ED00E000E100E008B50848084B0360E1
:102EA000B7234360002383600922C260036183610A
:102EB00004F0C4FE00B908BDFFF78AFE0804002034
:102EC0000044014008B50B480B4B03604FF4E1335D
:102ED000436000238360C36003610C22426183610D
:102EE000C3610362436207F0C0FD00B908BDFFF78C
:102EF0006FFE00BF34030020007C004000B589B0A5
:102F0000002304930593069307930193029303937D
:102F10001348144A0260436083605B22C26003610D
:102F20004361836104F08AFE98B94FF4805304939F
:102F300004A90B4804F0C4FF68B90023019302936D
:102F4000039301A9064805F04DF930B909B05DF8C1
:102F500004FBFFF73DFEFFF73BFEFFF739FE00BF26
:102F6000540400200004014000B589B000230193FF
:102F70000293039304930593069307931448154A09
:102F800002600122426083605B22C2600361802391
:102F9000836104F053FEA8B90D4804F07FFE98B990
:102FA000602301935B23029300220392059201A9FF
:102FB000074804F0DBFE48B9054801F0D3FA09B030
:102FC0005DF804FBFFF704FEFFF702FEFFF700FECB
:102FD000BC0300200048014000B58FB000230A93D5
:102FE0000B930C930D93079308930993009301930C
:102FF000029303930493059306931E481E4A0260AE
:10300000436083602D22C2600361836104F016FE79
:1030100030BB4FF480530A930AA9164804F050FFBE
:1030200000BB144804F03AFEF0B90023079309935B
:1030300007A9104805F0D6F8C0B9602300931623FD
:10304000019300230293049308226946094804F07F
:103050008DFE68B9074801F085FA0FB05DF804FBF2
:10306000FFF7B6FDFFF7B4FDFFF7B2FDFFF7B0FDC8
:10307000FFF7AEFDA00400200008004000B595B0A9
:103080003422002107A8FDF767FB00230293039376
:10309000049305930693244B1A6C42F080521A64F1
:1030A0001B6C03F080530093009B204B1A6842F482
:1030B00040421A601B6803F440430193019B0123C3
:1030C00007934FF48033089302230D934FF480024B
:1030D0000E9219220F924FF4B87210921193082297
:1030E0001292139307A801F03DFEB0B902F0A4FDBF
:1030F000A8B90F23029302230393002304934FF4F0
:10310000A05305934FF480530693062102A802F0C2
:103110009FF830B915B05DF804FBFFF759FDFFF7D4
:1031200057FDFFF755FD00BF00380240007000401A
:103130002DE9F0472DED028B82B002F057FEFFF72C
:103140009DFFFEF7A9FCFEF7ABF9FEF7C9FD00F005
:103150001DFEFEF767FFFEF7B3FFFFF73BFDFFF72E
:103160009DFDFEF727FEFEF78DFEFEF7F3FEFFF74F
:10317000CBFDFEF783F9FEF7EFFFFFF733F8FFF71C
:103180008BFEFFF79FFEFFF7B9FEFFF7EDFEFFF79F
:1031900023FFFFF76DF887496423CB62CB6A0133C5
:1031A0005B08013BCB63CB6A5B000133824AD3628D
:1031B000D36A01335B08013B5363CB6AD362D36AA2
:1031C00001335B08013B53634CE07C4B1B78002BC5
:1031D0004FD17B4A52E8003F43F4807342E800310C
:1031E0000029F6D1764A52E8003F43F0200342E836
:1031F00000310029F6D1724A02F1080353E8003F7A
:1032000043F00103083242E800310029F3D16D4B4D
:10321000002283F8252320225A60684B01221A706D
:1032200027E0694B00221A70684B5A681A61FEF752
:1032300023FC674B1B78022B00F04B84032B00F020
:103240007E84012B09D1634C02212046FFF78AFCC2
:103250000023237063705E4A13705F4B1B78012B51
:1032600000F06F844FF480715C4802F0CFFC0128BD
:10327000ABD05B4B1B78092BDBD801A252F823F0B3
:1032800023320008A932000813330008493300082C
:103290007933000889330008A53300080D3400088D
:1032A00061350008A73500084E4C0D212046FFF778
:1032B000C5FB4D4B18802046FFF7CCFB70B9454A43
:1032C000137843F004031370454B02221A703E4BEF
:1032D00000221A703E4B01221A70AAE7434A136873
:1032E00043F04003136002F58E32136843F040034D
:1032F00013603F4B3F4A40492046FFF723FA3F4BBC
:103300001A683F4B1A600723354A13702E4A137010
:10331000E0E72E4B5A681A61FEF7AEFBFEF7A8FFF6
:10332000324A136823F04003136002F58E321368AB
:1033300023F0400313600023294A1370224A1370BC
:10334000234B01221A7074E72E48FFF7C5FB82B2A7
:103350002D4B1A801F490B7803430B7042B91C4B4D
:1033600003221A700023184A13701D4A137060E775
:10337000174B01221A70F5E7154B02221A70124BF7
:103380001A78174B1A7054E7FFF7CCFB114A1378E1
:10339000034313700E4B01221A700B4B1A78104B1B
:1033A0001A7046E70A4B01221A70074B1A780C4B29
:1033B0001A703EE70008004000480140D702002094
:1033C0000010014000E100E0FF020020C0010020E9
:1033D000FE020020FC020020D90200200000024072
:1033E0000003002090020020D0020020003800409E
:1033F0002C02002060020020700200203003002018
:103400002C030020B0020020CE0200207A4B5A6824
:103410001A61FEF731FB794B1B68794A12689342B7
:103420007FF607AF764A13600120FEF715FA754F55
:1034300038810120FEF710FA38810220FEF70CFADD
:10344000714E30810220FEF707FA30810320FEF72B
:1034500003FA0320FEF700FA38800420FEF7FCF997
:103460000420FEF7F9F93080DFF8D08101223946D7
:103470004046FEF7EDF80146644D28800320FFF733
:10348000B5F8DFF8B491022231464846FEF7E0F87D
:10349000014628800420FFF7A9F83B895C4C638033
:1034A0003389A380B8F80C100120FFF79FF8B9F812
:1034B0000C100220FFF79AF80020FFF75FF8288031
:1034C0000120FFF75BF82880E0810120FFF756F824
:1034D000288020820120FFF751F828806082012097
:1034E000FFF74CF82880A0820120FFF747F82880DA
:1034F000E0820220FFF742F828800320FFF73EF821
:1035000028800420FFF73AF8288020830520FFF761
:1035100035F828803F4B1B683F4A1360E3801B0C43
:1035200023813B8863813388A3813C4BDB7A012B69
:1035300003D03B4B07221A707BE602340D21204654
:10354000FFF77CFA0346374A1080A01E8383FFF7FB
:10355000A5FA0346288034490A7813430B70E8E73C
:103560003248FFF777FA70B92F4A137843F0040313
:1035700013702F4B02221A70294B00221A702D4B08
:1035800001221A7055E6254B2B4A2C492748FDF796
:10359000ABFF204B1A682A4B1A600923244A137088
:1035A0001F4A1370EBE7144B1B78012B54D0022BEE
:1035B00000F08E81114B1B68114A1268934200F291
:1035C0003582204B1B78002BFBD0FEF755FA0A4BB7
:1035D000DB8A032B0BD91C4B1A681C4BDA60064B99
:1035E0001B7D1B4AA2FB0323DB081A4A13600C4B0A
:1035F00009221A701DE600BFC00100201803002038
:10360000140300200C02002000020020CE02002043
:10361000B002002030030020280300202C020020EC
:10362000FF020020D0020020FC02002090020020B7
:1036300000030020FE020020600200207002002033
:103640002C030020D60200200403002008040020E0
:10365000CDCCCCCC080300208B4BD3ED077AFCEE0D
:10366000E77A17EE903A99B20220FEF7BFFF0320E7
:10367000FEF7F2F80320FEF7EFF8844C20800420D8
:10368000FEF7EAF80420FEF7E7F8814D28800122D2
:1036900021468048FDF7DCFF01467F4C2080032057
:1036A000FEF7A4FF022229467C48FDF7D1FF014620
:1036B00020800420FEF79AFF01228021784802F042
:1036C000ACFA784804F006F9002840F097806E4D77
:1036D00095ED027AD5ED047A37EE677AD5ED036A77
:1036E000C7EE267AB2EE047A67EE877AFCEEE77AC6
:1036F000CDED017A9DF80470DFF8CCA10021504691
:1037000004F01AFDDFF8C4910821484604F014FDC6
:10371000DFF8A881D8F8003023F00803C8F800309B
:10372000614E336823F0080333600024C8F8244056
:1037300074622146504604F053FC0821484604F0C8
:103740004FFCF36A143B7362C8F8244095ED026A9B
:10375000D5ED047A36EE676AB7EEC66AB0EE085B5E
:1037600086EE057B95ED036AB7EEC66A87EE065BCB
:10377000FCEEC58B37EE077B87EE065BBCEEC58B98
:103780002546414BD3ED047A93ED027AF4EEC77AE5
:10379000F1EE10FA45D5454B1B78002BF1D0FCEE2D
:1037A000E77A17EE903A99B20120FEF71FFF4FF427
:1037B00000713F4802F037FA334BD3ED047A93EDB2
:1037C000037A77EE877AC3ED047A0023394A1360CF
:1037D000364A137018EE903A8BB118EE103AA3B136
:1037E000B4FBF7F307FB13439BB2A3B10134A4B2BC
:1037F000002280212A4802F010FAC2E7FEE70122E7
:1038000010212D4802F009FAE7E7012220212A4879
:1038100002F003FAE4E7E8B2FDF78CFF0135ADB240
:10382000E4E7264AD36843F00103D360FEF724F9A6
:10383000214C00221021204602F0EFF90022202125
:10384000204602F0EAF9104CD4ED017AC4ED047A76
:10385000FCEEE77A17EE903A99B20120FEF7C6FE29
:10386000E38A032B0CD90F4AD0681549086042F24D
:103870000F71D160013B642202FB03F3114A136014
:10388000084804F027F895E6C00100200C0200204B
:103890000002002070020020CE0200206002002002
:1038A000000C02400804002000080040D60200205E
:1038B000001802400C0300200004024000480140B0
:1038C0000403002008030020BC030020A004002003
:1038D000A74BD3ED077AFCEEE77A17EE903A99B250
:1038E0000120FEF783FE0320FDF7B6FF0320FDF75E
:1038F000B3FFA04C20800420FDF7AEFF0420FDF7AD
:10390000ABFF9D4D2880012221469C48FDF7A0FE7B
:1039100001469B4C20800320FEF768FE02222946C8
:103920009848FDF795FE014620800420FEF75EFED4
:10393000954B02221A7000229A721A814FF47A7201
:103940001A81924A5A6080225A80914B42F2107238
:10395000DA62904803F0BEFF78BB012280218E48D6
:1039600002F05BF942F21073013BFDD1002280218D
:10397000894802F052F9844B02229A72874803F078
:10398000A9FFD8B97A4BD3ED047A93ED027AF4EE1D
:10399000C77AF1EE10FA12D5814B1B78002BF1D0CB
:1039A000734B93ED037A77EE277AC3ED047A002305
:1039B0007C4A13607A4A1370E4E7FEE7FEE7774833
:1039C00003F073FF744C01228021204602F025F998
:1039D00000228021204602F020F96E4803F0C2FF49
:1039E0006B4B00225A62FEF747F8614CD4ED017A26
:1039F000C4ED047AFCEEE77A17EE903A99B2022011
:103A0000FEF7F4FDE38A032B0CD9644AD0686649BB
:103A1000086042F20F71D160013B642202FB03F3A4
:103A2000624A13605D4803F055FFC3E5604A1360C6
:103A30000120FDF711FF4F4E30810120FDF70CFFF3
:103A400030810220FDF708FF4B4F38810220FDF73F
:103A500003FF38813389574C6380A0800020FEF734
:103A60008DFD474D28800120FEF788FD2880E081EC
:103A70000120FEF783FD288020820120FEF77EFDD5
:103A8000288060820120FEF779FD2880A082012035
:103A9000FEF774FD2880E0820220FEF76FFD28808B
:103AA0000320FEF76BFD28800420FEF767FD2880C9
:103AB00020830520FEF762FD28803F4B1B683F4AAC
:103AC0001360E3801B0C2381338863813B88A381CF
:103AD00077E53B4C0D212046FEF7B0FF394B1880AF
:103AE000608300230BE0334A32F813205900364834
:103AF00000F813200131120A425401339BB20E2BFD
:103B0000F1D91E20FFF744F8304B00221A70FFF75E
:103B1000A4BB284A32F8132059002B4800F8132080
:103B20000131120A425401339BB20E2BF1D91E20EF
:103B3000FFF72EF8254B00221A70FFF78EBB0023EB
:103B4000F3E71D4B1B68224A12689B1A642B7FF611
:103B500089AB00221F4B1A801F490B7843F00203E8
:103B60000B701A4B012119701C4B1A70FFF77ABBAE
:103B7000C00100200C020020000200207002002082
:103B8000CE02002060020020F40100200004024068
:103B90000004014054040020000C024008040020EE
:103BA000D60200200C03002004030020080300209C
:103BB00014030020B002002030030020280300205E
:103BC000B2020020D0020020DC020020FE02002011
:103BD00024030020D4020020FC020020D90200208F
:103BE00000B583B0009313460A460146034803F02C
:103BF00089F800B1012003B05DF804FBEC0400205B
:103C000000B583B0009313460A460146034803F00B
:103C10009DF900B1012003B05DF804FBEC04002025
:103C200008B5034803F0D0FC043818BF012008BDD4
:103C3000EC04002008B50146014803F052FC08BD21
:103C4000EC04002000B583B001238DF8073000F0AC
:103C5000ADF810B900238DF807309DF8070003B0C8
:103C60005DF804FB38B5FFF7EDFF012802D002250F
:103C7000284638BD0446074803F018FC05460028CE
:103C8000F6D14FF40061034803F03EFC0028EFD06A
:103C90002546EDE7EC04002008B5074B01221A7019
:103CA000FFF7BEFF20B9044A137803F0FE03137038
:103CB000014B187808BD00BF5000002010B5044625
:103CC000074B01221A70FFF7CDFF10B1044B187893
:103CD00010BD2046FFF7E0FF014B1870F6E700BF6C
:103CE0005000002008B5FFF7D7FF08BD08B508460B
:103CF00011461A464FF0FF33FFF772FF30B9FFF756
:103D00008FFF03460028FAD1184608BD0123FBE7C0
:103D100008B5084611461A464FF0FF33FFF770FF0B
:103D200030B9FFF77DFF03460028FAD1184608BDD9
:103D30000123FBE730B589B0134B187810F001046C
:103D40001BD1154603291CD8DFE801F002040A1034
:103D50000C4613E06846FFF76DFF069B2B600DE0F5
:103D60006846FFF767FF079B2B8007E06846FFF771
:103D700061FF079B5B0A2B6000E00324204609B02B
:103D800030BD0424FAE700BF5000002008B5034905
:103D9000034806F067FB034B187008BD00060020BF
:103DA000E8AC0008040600200020704708B5012197
:103DB000034801F02BFF08B9012008BD0020FCE7F3
:103DC000000C0240FEE7FEE7FEE7FEE7FEE7704775
:103DD0007047704708B502F015F808BD08B50348EC
:103DE00000F031FE024800F02EFE08BDB8050020AC
:103DF0007005002008B5084A136801331360074AAC
:103E00001268934203D0064803F0CBFD08BD054B72
:103E100001221A70F7E700BF0C03002008030020FE
:103E200008040020D602002008B5094B1A6842F0A9
:103E300008021A6007490A6842F008020A60DA6854
:103E400022F00102DA60044803F0ABFD08BD00BFB8
:103E50000048014000080040BC03002070470000FB
:103E600010B5114B9B7A022B0ED0032B18D10021D9
:103E70000220FEF7BBFB0C4C00226188606801F059
:103E8000CCFE0223A3720BE0074C21890220FEF72F
:103E9000ADFB01226188606801F0BFFE0323A372BD
:103EA000024803F07EFD10BDF40100205404002000
:103EB0007047000008B5094B1B6913F0010F0BD0C8
:103EC000064B6FF001021A61054A13680133136053
:103ED0000221044801F0A7FE08BD00BF0010004009
:103EE00030030020000C0240064B1B6913F0010F49
:103EF00007D0044B6FF001021A61034A13680133C3
:103F000013607047001400401803002010B4974B52
:103F10005A6AD2B2964B1A70964B1B881F2B00F22E
:103F20000B81DFE813F020002F00090109010901CE
:103F30000901090109010901090109010901090131
:103F40000901090109010901090109010901090121
:103F50000901090109010901090109010901090111
:103F600095000901CF0084490868844908608449A4
:103F70000120087083490A8003447E4A13805DF85B
:103F8000044B70477F490B8803EB02239BB20B80E5
:103F900044F24442934237D00FD842F22222934255
:103FA00020D043F23332934225D041F21112934292
:103FB00040D1704B02221A80E1E746F266629342DA
:103FC0002BD047F27772934230D045F2555293424C
:103FD00030D10023674A1380694A13706A4B052267
:103FE0001A70CCE70023634A1380654A1370664B4E
:103FF00002221A70C3E700235E4A1380604A1370DE
:10400000614B03221A70BAE700235A4A13805C4AB4
:1040100013705D4B04221A70B1E70023554A1380D8
:10402000574A1370584B06221A70A8E7514B0222C8
:104030001A80A4E700234F4A1380514A1370534A51
:10404000137843F0020313704F4B02221A7096E765
:104050004C49088841F21111884212D013F0010F27
:104060002AD0590801394A4C34F8110000EB0222D9
:1040700024F8112001333F4A1380464B00221A7066
:104080007DE713F0010F11D05B08013B404830F889
:10409000131001EB022220F813203B4B01221A706F
:1040A0000023344A1380364A137068E75B08013BEB
:1040B000374921F81320F0E759080139344820F82E
:1040C0001120D7E72F49088847F27771884212D02C
:1040D00013F0010F2AD0590801392D4C34F8110082
:1040E00000EB022224F811200133224A1380294BCD
:1040F00000221A7043E713F0010F11D05B08013B57
:10410000234830F8131001EB022220F813201E4B35
:1041100008221A700023174A1380194A13702EE7D9
:104120005B08013B1A4921F81320F0E759080139CF
:10413000174820F81120D7E713F0010F0FD05908C6
:104140000139134C34F8110000EB022224F811203D
:104150000133084A13800F4B00221A700FE75908E9
:1041600001390B4820F81120F2E700BF0010014090
:1041700001030020D402002030030020240300208B
:10418000D9020020D202002000030020FC020020FF
:1041900090020020FE02002000B583B0304BDB69A6
:1041A00013F0200F07D02E4B1B6813F0200F02D006
:1041B000FFF7ACFE33E02A4BDB6913F0080F25D183
:1041C000274BDB6913F0020F2CD1254BDB6913F071
:1041D000040F31D1224BDB6913F0010F36D1214B93
:1041E000DB6913F0400F1AD01E4B1B6813F0400F11
:1041F00015D01B4B40221A62194A52E8003F23F0A7
:10420000400342E800310029F6D108E0144B5B6A14
:104210009DF8072052FA83F3DBB28DF8073003B024
:104220005DF804FB0E4B5B6A9DF8072052FA83F39E
:10423000DBB28DF80730F2E7094B5B6A9DF8072087
:1042400052FA83F3DBB28DF80730E8E7044B5B6A80
:104250009DF8072052FA83F3DBB28DF80730DEE7D2
:104260000010014000140140024B4FF00062DA6080
:10427000704700BF0064024008B50A4B5B6813F04A
:10428000006F09D1074B5B6813F0007F03D0054B2B
:104290004FF00072DA6008BDFFF7E6FF024B002224
:1042A0001A70F8E700640240D802002082B00A4B7E
:1042B0001A6C42F080521A641A6C02F0805200921A
:1042C000009A5A6C42F480425A645B6C03F4804357
:1042D0000193019B02B070470038024030B58DB0A9
:1042E00000230793089309930A930B930368384AB2
:1042F000934204D0374A934246D00DB030BD364B7E
:104300005A6C42F480725A645A6C02F480720192C0
:10431000019A1A6B42F004021A631A6B02F004024B
:104320000292029A1A6B42F001021A631A6B02F0AF
:1043300001020392039A1A6B42F002021A631B6B8A
:1043400003F002030493049B03240794089407A931
:10435000224801F059FB042307930894002509958E
:1043600007A91F4801F050FB07940894099507A975
:104370001C4801F049FB2A462946122001F0DEFCC8
:10438000122001F0EBFCB8E7134B5A6C42F4806248
:104390005A645A6C02F480620592059A1A6B42F0D4
:1043A00020021A631B6B03F020030693069B202355
:1043B00007930323089307A90B4801F025FB00226C
:1043C0001146122001F0BAFC122001F0C7FC94E75C
:1043D0000020014000220140003802400008024055
:1043E000000002400004024000140240F0B5ADB0ED
:1043F000044600212791289129912A912B919022FE
:1044000003A8FCF7A9F92268224B9A4201D02DB0EB
:10441000F0BD4FF42003039303A800F0F5FF00283C
:1044200035D11D4B5A6C42F400625A645A6C02F446
:1044300000620092009A1A6B42F004021A631A6B2F
:1044400002F004020192019A1A6B42F008021A6308
:104450001B6B03F008030293029B4FF4F85327935E
:10446000022728970026299603252A950C242B94A9
:1044700027A90A4801F0C8FA042327932897299608
:104480002A952B9427A9064801F0BEFABFE7FEF74C
:104490009FFBC6E7002C01400038024000080240A4
:1044A000000C024000B585B00368294A93420BD046
:1044B000284A934213D0284A934223D0274A934252
:1044C00033D005B05DF804FB254B1A6C42F00402B2
:1044D0001A641B6C03F004030093009BF1E7204B6C
:1044E0005A6C42F002025A645B6C03F002030193BF
:1044F000019B002211462C2001F020FC2C2001F011
:104500002DFCDEE7164B5A6C42F400325A645B6CA9
:1045100003F400330293029B00221146192001F09C
:104520000DFC192001F01AFCCBE70D4B5A6C42F43C
:1045300080225A645B6C03F480230393039B002264
:1045400011461A2001F0FAFB1A2001F007FCB8E727
:1045500000080040000401400044014000480140C0
:104560000038024000B589B00023039304930593FB
:104570000693079303681A4A934205D0194A934257
:1045800017D009B05DF804FB174B1A6B42F002021A
:104590001A631B6B03F002030193019B4FF48073BA
:1045A000039302230493079303A9104801F02CFA04
:1045B000E7E70D4B1A6B42F002021A631B6B03F024
:1045C00002030293029B4FF40073039302230493AC
:1045D0000323079303A9054801F016FAD1E700BFAA
:1045E000000800400048014000380240000402403A
:1045F00010B5ACB0044600212791289129912A9149
:104600002B91902203A8FCF7A7F82268174B9A4237
:1046100001D02CB010BD4FF40053039303A800F059
:10462000F3FE00BB124B1A6C42F000421A641A6C83
:1046300002F000420192019A1A6B42F010021A63D2
:104640001B6B03F010030293029B032327930222A8
:104650002892002229922A9308232B9327A9054800
:1046600001F0D2F9D5E7FEF7B3FADBE7007C0040B2
:1046700000380240001002404A4B5A6822F440328F
:104680005A605A6841680A435A600268536823F4C2
:104690008073536002685368016943EA01235360E1
:1046A0000268536823F0407353600268536881685E
:1046B0000B4353600268936823F4006393600268BD
:1046C0009368C1680B439360826A374B9A4257D014
:1046D0000268936823F07063936002689368816A4C
:1046E0000B4393600268936823F040539360026821
:1046F0009368C16A0B4393600268936823F00203D6
:10470000936002689368816943EA4103936090F87B
:104710002030002B3FD00268536843F4006353609D
:104720000268536823F46043536001684B68426A2F
:10473000013A43EA42334B600268D36A23F47003C0
:10474000D3620168CB6AC269013A43EA0253CB6281
:104750000268936823F4007393600268936890F88A
:10476000301043EA412393600268936823F4806326
:10477000936002689368416943EA812393607047BC
:104780000268936823F0706393600268936823F073
:1047900040539360B0E70268536823F400635360AA
:1047A000CAE700BF002301400100000F28B310B585
:1047B0000446036C43B1236C13F0100F0BD001209F
:1047C000002384F83C3010BDFFF788FD00236364AC
:1047D00084F83C30EFE7226C094B134043F00203AE
:1047E00023642046FFF748FF00206064236C23F019
:1047F000030343F001032364E2E70120704700BF95
:10480000FDEEFFFF82B00023019390F83C30012BB6
:104810007ED0012380F83C3003689A6812F0010FC3
:1048200013D19A6842F001029A603D4B1B683D4AE1
:10483000A2FB03239B0C03EB4303019302E0019BC8
:10484000013B0193019B002BF9D103689A6812F098
:10485000010F52D0016C344A0A4042F48072026463
:104860005A6812F4806F05D0026C22F4405242F470
:1048700080520264026C12F4805F19D0426C22F004
:1048800006024264002280F83C206FF022021A6087
:10489000264B5B6813F01F0F0DD103689A6812F066
:1048A000405F37D19A6842F080429A6000202DE044
:1048B00000224264E6E703681D4A93420AD01B4B7C
:1048C0005B6813F0100F27D103681A4A93420AD08D
:1048D00000201BE09A6812F0405FF0D19A6842F025
:1048E00080429A60EBE79A6812F0405F16D19A68AE
:1048F00042F080429A60002008E0036C43F010030D
:104900000364436C43F001034364002002B070472A
:104910000220FBE70020F9E70020F7E70020F5E799
:104920005800002083DE1B43FEF8FFFF00230140F8
:10493000002001400022014090F83C30012B17D0AC
:10494000012380F83C300268936823F001039360F0
:1049500003689B6813F0010F05D1026C054B1340EF
:1049600043F001030364002380F83C30184670478D
:1049700002207047FEEEFFFF70B504460D46036847
:104980009A6812F4806F03D09B6813F4807F19D16A
:1049900001F044FA064623681A6812F0020F20D18B
:1049A000B5F1FF3FF7D0B5B923681B6813F0020FCC
:1049B000F1D1236C43F004032364002384F83C30DA
:1049C000032033E0036C43F020030364002380F8EA
:1049D0003C3001202AE001F021FA801BA842DAD9FC
:1049E000E2E76FF012021A60236C43F40073236451
:1049F00023689A6812F0405F17D1A269BAB9DA6ADF
:104A000012F4700F03D09B6813F4806F11D1236CE4
:104A100023F480732364236C13F4805F0BD1236C25
:104A200043F001032364002000E0002070BD00205B
:104A3000FCE70020FAE70020F8E70368D86C70472D
:104A400070477047704770B5044603681E685D681C
:104A5000C5F3401212EA56022CD0026C12F0100F6D
:104A600003D1026C42F4007202649A6812F0405F53
:104A700019D1A269BAB9DA6A12F4700F03D09A6830
:104A800012F4806F0FD15A6822F020025A60236C12
:104A900023F480732364236C13F4805F03D1236CAD
:104AA00043F0010323642046FFF7CAFF23686FF039
:104AB00012021A60C5F3C01313EA960335D0236CB3
:104AC00013F0100F03D1236C43F4005323642368C5
:104AD0009A6812F4401F21D19A6B12F4401F03D040
:104AE0009A6812F4806F19D15A6812F4806F15D148
:104AF0009A6812F0405F11D1A2697AB95A6822F01F
:104B000080025A60236C23F480532364236C13F4D3
:104B1000807F03D1236C43F001032364204600F01F
:104B20001FF923686FF00C021A60C5F380131E4250
:104B300004D023681B6813F0010F05D1C5F380650D
:104B400015EA56150CD170BD236C43F480332364F1
:104B50002046FFF776FF23686FF001021A60EDE749
:104B6000636C43F00203636423686FF020051D60EB
:104B70002046FFF767FF23681D60E4E730B482B08A
:104B80000022019290F83C20012A00F0DC800346CC
:104B9000012280F83C200A68B2F1004F18BF092AB0
:104BA00022D90468E06892B202EB42021E3A4FF04A
:104BB000070C0CFA02F220EA0202E2600A6863487B
:104BC00082420AD01D68E8688C6892B202EB420209
:104BD0001E3A94402043E8601CE01868C2688C6864
:104BE00042EA0462C26015E00468206992B202EBF6
:104BF00042024FF0070C0CFA02F220EA0202226194
:104C00001C6820690A8802EB42028D6805FA02F2EC
:104C1000024322614A68062A29D81C68606B02EBAD
:104C20008202053A4FF01F0C0CFA02F220EA02024F
:104C300062631C68606B4A6802EB8202053AB1F855
:104C400000C00CFA02F2024362631868404A9042C4
:104C50003DD018683E4A904243D018683C4A904282
:104C60004CD0002083F83C0002B030BC70470C2AC6
:104C700016D81D68286B02EB8202233A1F2404FA1F
:104C800002F220EA02022A631D68286B4A6802EBDE
:104C90008202233A0C8804FA02F202432A63D4E720
:104CA0001D68E86A02EB8202413A1F2404FA02F20C
:104CB00020EA0202EA621D68E86A4A6802EB8202A0
:104CC000413A0C8804FA02F20243EA62BDE70A683C
:104CD000B2F1004FBDD11F48426822F44002426049
:104CE000B7E70A68122AB8D11A4A506820F40000BF
:104CF0005060506840F480005060AEE70A68134886
:104D0000112A18BF8242ACD1124A506820F48000A8
:104D10005060506840F40000506009680B4A9142AE
:104D20009FD10D4A12680D49A1FB0212920C02EBB1
:104D300082025200019202E0019A013A0192019A24
:104D4000002AF9D18DE702208EE700BF1200001083
:104D500000200140002301405800002083DE1B4357
:104D600070470000002800F0068270B582B004464B
:104D7000036813F0010F29D0954B9B6803F00C03D7
:104D8000042B1AD0924B9B6803F00C03082B0FD016
:104D90006368B3F5803F40D0002B54D18C4B1A6828
:104DA00022F480321A601A6822F480221A6039E0F4
:104DB000874B5B6813F4800FEAD0854B1B6813F4B4
:104DC000003F03D06368002B00F0D781236813F005
:104DD000020F74D07E4B9B6813F00C0F5ED07C4B9F
:104DE0009B6803F00C03082B53D0E368002B00F002
:104DF0008980774A136843F00103136001F00EF8CD
:104E00000546734B1B6813F0020F72D101F006F8D0
:104E1000401B0228F5D90320B4E16D4A136843F41E
:104E20008033136063682BB300F0F8FF0546684BCE
:104E30001B6813F4003FC9D100F0F0FF401B642849
:104E4000F5D903209EE1B3F5A02F09D0604B1A6875
:104E500022F480321A601A6822F480221A60E1E794
:104E60005B4B1A6842F480221A601A6842F480325E
:104E70001A60D7E700F0D2FF0546554B1B6813F4C4
:104E8000003FA3D000F0CAFF401B6428F5D90320DF
:104E900078E14F4B5B6813F4800FA6D14C4B1B6835
:104EA00013F0020F03D0E368012B40F06881484AF9
:104EB000136823F0F803216943EAC10313602368F0
:104EC00013F0080F46D0636983B3414A536F43F030
:104ED0000103536700F0A2FF05463D4B5B6F13F0E3
:104EE000020F37D100F09AFF401B0228F5D90320AA
:104EF00048E1374A136823F0F803216943EAC10304
:104F00001360DCE7324A136823F00103136000F0FA
:104F100085FF05462E4B1B6813F0020FCFD000F023
:104F20007DFF401B0228F5D903202BE1284A536F4F
:104F300023F00103536700F071FF0546244B5B6FBC
:104F400013F0020F06D000F069FF401B0228F5D9CC
:104F5000032017E1236813F0040F7DD01C4B1B6C5A
:104F600013F0805F1ED11A4B1A6C42F080521A6403
:104F70001B6C03F080530193019B0125154B1B68AB
:104F800013F4807F10D0A368012B25D0002B3BD1D8
:104F90000F4B1A6F22F001021A671A6F22F00402F7
:104FA0001A671EE00025E9E70A4A136843F4807394
:104FB000136000F033FF0646064B1B6813F4807F36
:104FC000E1D100F02BFF801B6428F5D90320D9E044
:104FD0000038024000700040724A136F43F0010332
:104FE0001367A36833B300F019FF06466D4B1B6FC0
:104FF00013F0020F2FD100F011FF801B41F2883314
:105000009842F3D90320BDE0052B09D0654B1A6FF8
:1050100022F001021A671A6F22F004021A67E0E711
:10502000604B1A6F42F004021A671A6F42F00102D5
:105030001A67D6E700F0F2FE06465A4B1B6F13F0D4
:10504000020F08D000F0EAFE801B41F2883398423C
:10505000F3D9032096E0FDB9A369002B00F09180FD
:10506000504A926802F00C02082A59D0022B19D03B
:105070004C4A136823F08073136000F0CFFE04469F
:10508000484B1B6813F0007F48D000F0C7FE001BA0
:105090000228F5D9032075E0424A136C23F08053AF
:1050A0001364D9E73F4A136823F08073136000F05C
:1050B000B5FE05463B4B1B6813F0007F06D000F0A1
:1050C000ADFE401B0228F5D903205BE0E369226AAC
:1050D0001343626A43EA8213A26A5208013A43EA1E
:1050E0000243E26A43EA0263226B43EA02732D4AF7
:1050F0005360136843F08073136000F08FFE044622
:10510000284B1B6813F0007F06D100F087FE001BC0
:105110000228F5D9032035E0002033E0002031E0FB
:10512000204A5268012B2FD002F48003E1698B42A0
:105130002CD102F03F03216A8B4229D1616A47F6E4
:10514000C0731340B3EB811F24D102F44031A36A32
:105150005B08013BB1EB034F1ED102F07063E16AC3
:10516000B3EB016F1AD102F0E042236BB2EB037F85
:1051700016D1002006E001207047012002E0012046
:1051800000E0002002B070BD0120FBE70120F9E73C
:105190000120F7E70120F5E70120F3E70120F1E71F
:1051A0000120EFE70038024008B5264B9B6803F06A
:1051B0000C03042B41D0082B41D1224B5A6802F03A
:1051C0003F025B6813F4800F12D01E4B5968C1F385
:1051D00088111D480023A1FB0001FBF7B7FF194B05
:1051E0005B68C3F3014301335B00B0FBF3F008BD20
:1051F000144B5868C0F388104FEA401CBCEB000CFD
:105200006EEB0E0E4FEA8E1343EA9C634FEA8C114D
:10521000B1EB0C0163EB0E03DB0043EA5173C900F1
:1052200011EB000C43F10003990200234FEA8C209C
:1052300041EA9C51FBF78AFFD1E70348D7E70348CF
:10524000D5E700BF0038024040787D010024F4001B
:10525000002800F0A08070B50D460446524B1B6834
:1052600003F00F038B420BD24F4A136823F00F0356
:105270000B431360136803F00F038B4240F08D80E3
:10528000236813F0020F17D013F0040F04D0474A1D
:10529000936843F4E0539360236813F0080F04D03D
:1052A000424A936843F460439360404A936823F012
:1052B000F003A1680B439360236813F0010F31D012
:1052C0006368012B20D0022B25D0384A126812F0D7
:1052D000020F64D035498A6822F0030213438B60C1
:1052E00000F09CFD0646314B9B6803F00C0362689E
:1052F000B3EB820F16D000F091FD801B41F2883392
:105300009842F0D9032045E0284A126812F4003F81
:10531000E0D101203EE0254A126812F0007FD9D189
:10532000012037E0204B1B6803F00F03AB420AD982
:105330001D4A136823F00F032B431360136803F017
:105340000F03AB422DD1236813F0040F06D0174A88
:10535000936823F4E053E1680B439360236813F0F0
:10536000080F07D0114A936823F46043216943EA88
:10537000C1039360FFF718FF0C4B9B68C3F3031343
:105380000B4AD35CD8400B4B18600B4B186800F0ED
:1053900007FD002070BD012070470120FAE70120C1
:1053A000F8E70120F6E700BF003C02400038024069
:1053B00004AD00085800002054000020014B18687C
:1053C000704700BF5800002008B5FFF7F7FF044BF7
:1053D0009B68C3F38223034AD35CD84008BD00BF57
:1053E00000380240FCAC000808B5FFF7E7FF044BAB
:1053F0009B68C3F34233034AD35CD84008BD00BF67
:1054000000380240FCAC0008F0B583B004460668E2
:1054100016F001060DD0B54B9A6822F400029A608E
:105420009A68416B0A439A60436B002B00F06781D6
:105430000026256815F4002511D0AC4AD2F88C302E
:1054400023F44013E16B0B43C2F88C30E36BB3F5EC
:10545000801F00F05681002B00F055810025236845
:1054600013F4801F0FD0A14AD2F88C3023F44003EC
:10547000216C0B43C2F88C30236CB3F5800F00F025
:10548000448103B90125236813F0807F00D00126F1
:1054900013F0200F40F03B81236813F0100F0CD065
:1054A000924BD3F88C2022F08072C3F88C20D3F872
:1054B0008C20A16B0A43C3F88C20236813F4804F1F
:1054C00008D08A4AD2F8903023F44033616E0B43FF
:1054D000C2F89030236813F4004F08D0834AD2F802
:1054E000903023F44023A16E0B43C2F89030236820
:1054F00013F4803F08D07D4AD2F8903023F4401353
:10550000E16E0B43C2F89030236813F4003F08D0DB
:10551000764AD2F8903023F44003216F0B43C2F84F
:105520009030236813F0400F08D0704AD2F89030C2
:1055300023F00303616C0B43C2F89030236813F02F
:10554000800F08D0694AD2F8903023F00C03A16C88
:105550000B43C2F89030236813F4807F08D0634A6D
:10556000D2F8903023F03003E16C0B43C2F8903056
:10557000236813F4007F08D05C4AD2F8903023F0FF
:10558000C003216D0B43C2F89030236813F4806F81
:1055900008D0564AD2F8903023F44073616D0B4323
:1055A000C2F89030236813F4006F08D04F4AD2F845
:1055B000903023F44063A16D0B43C2F89030236810
:1055C00013F4805F08D0494AD2F8903023F4405356
:1055D000E16D0B43C2F89030236813F4005F08D0EC
:1055E000424AD2F8903023F44043216E0B43C2F874
:1055F0009030236813F4800F08D03C4AD2F89030E2
:1056000023F08063A16F0B43C2F89030236813F43A
:10561000001F0DD0354AD2F8903023F00063E16FBF
:105620000B43C2F89030E36FB3F1006F00F0D58008
:10563000236813F0080F00D0012513F4802F08D041
:105640002A4AD2F8903023F04073616F0B43C2F8BE
:105650009030236813F4000F09D0244AD2F8903018
:1056600023F08053D4F880100B43C2F890302368A5
:1056700013F0806F09D01D4AD2F8903023F0005308
:10568000D4F884100B43C2F89030236813F0006FF5
:1056900009D0164AD2F88C3023F00073D4F8881061
:1056A0000B43C2F88C30236813F0805F09D00F4A97
:1056B000D2F88C3023F08063D4F88C100B43C2F8FE
:1056C0008C3026B9236813F0007F00F00681074A6A
:1056D000136823F08063136000F0A0FB0646034BC1
:1056E0001B6813F0006F7AD002E000BF0038024060
:1056F00000F094FB801B6428F1D90320F0E0012620
:1057000097E60126A7E60125A9E60126B9E67F4B23
:105710001A6C42F080521A641B6C03F080530193A0
:10572000019B7B4A136843F48073136000F076FB9F
:105730000746774B1B6813F4807F06D100F06EFBA1
:10574000C01B6428F5D90320CAE0704B1B6F13F40B
:10575000407315D0226B02F440729A4210D06B4B0A
:105760001A6F22F44072196F41F480311967196F72
:1057700021F4803119671A671B6F13F0010F12D1E2
:10578000236B03F44072B2F5407F1DD05F4A9368EB
:1057900023F4F81393605D490B6F226BC2F30B0285
:1057A00013430B6778E600F039FB0746574B1B6F36
:1057B00013F0020FE4D100F031FBC01B41F288333B
:1057C0009842F3D903208BE05048826822F4F81203
:1057D000504919400A438260DDE7012528E7236824
:1057E00013F0010F13D0636B8BB9484AD2F88430A1
:1057F000D2F88410606803F4403343EA801301F068
:1058000070610B43A16843EA0173C2F884302368D6
:1058100013F4002F03D0E26BB2F5801F06D013F40F
:10582000801F1ED0236CB3F5800F1AD1374AD2F8EF
:105830008430D2F88410606803F4403343EA801364
:10584000E06843EA006301F0E0410B43C2F88430B2
:10585000D2F88C3023F01F03616A01390B43C2F880
:105860008C30236813F0807F11D0284AD2F884004E
:10587000D2F88410666823691B0443EA861300F09B
:105880007060034301F0E0410B43C2F884302368A9
:1058900013F0007F0DD0626823691B0443EA821372
:1058A000E26843EA0263A26843EA0273174AC2F855
:1058B0008430164A136843F08063136000F0AEFA38
:1058C0000646124B1B6813F0006F06D100F0A6FAD3
:1058D000801B6428F5D9032002E0012D02D00020AE
:1058E00003B0F0BD094A136823F08053136000F041
:1058F00095FA0546054B1B6813F0005F0CD000F0CD
:105900008DFA401B6428F5D90320E9E700380240EE
:1059100000700040FFFCFF0F236813F4002F01D03C
:10592000E26B22B113F4801F1DD0236CDBB9354A22
:10593000D2F88830D2F88810606903F4403343EA23
:105940008013A06943EA006301F0E0410B43C2F811
:105950008830D2F88C3023F4F853A16A013943EA35
:105960000123C2F88C30236813F4001F03D0E36FC7
:10597000B3F1006F31D0236813F0080F19D0214A1A
:10598000D2F88810D2F88830606903F4403343EAD3
:10599000801301F070610B43E16943EA0173C2F8BF
:1059A0008830D2F88C3023F44033E16A0B43C2F8DC
:1059B0008C30144A136843F08053136000F02EFAC1
:1059C0000446104B1B6813F0005F19D100F026FA53
:1059D000001B6428F5D9032082E70A4AD2F8880020
:1059E000D2F888106569236A1B0443EA851300F026
:1059F0007060034301F0E0410B43C2F88830BAE71E
:105A000000206DE70038024000230F2B00F2F480E5
:105A100070B582B066E085684FEA430E032404FA4D
:105A20000EF425EA0405CC6804FA0EF42C438460D5
:105A3000446824EA02044A68C2F300129A402243EE
:105A400042605DE0DC08083450F8242003F00705CC
:105A5000AD004FF00F0E0EFA05FE22EA0E0E0A6997
:105A6000AA4042EA0E0240F824205DE0092200E04C
:105A7000002202FA0EF22A430234604D45F8242037
:105A80005F4A94686FEA0C0224EA0C054E6816F42B
:105A9000801F01D04CEA0405594CA560E46802EA75
:105AA00004054E6816F4001F01D04CEA0405544C5E
:105AB000E560646802EA04054E6816F4003F01D010
:105AC0004CEA04054E4C6560246822404D6815F48C
:105AD000803F01D04CEA0402494C226001330F2B75
:105AE00000F2888001229A400C6804EA020C32EA33
:105AF0000404F3D14C6804F00304013C012C8AD95E
:105B00004A6802F00302032A09D0C4685D00032238
:105B1000AA4024EA02048A68AA402243C2604A6872
:105B200002F00302022A8DD004684FEA430E0322DA
:105B300002FA0EF224EA02044A6802F0030202FAB0
:105B40000EF2224302604A6812F4403FC6D02D4A4A
:105B5000546C44F480445464526C02F480420192C8
:105B6000019A9C08A51C254A52F8255003F0030E03
:105B70004FEA8E0E0F2202FA0EF225EA0205224AA1
:105B800090423FF475AF02F58062904222D002F558
:105B90008062904220D002F5806290421ED002F5D1
:105BA000806290421CD002F5806290421AD002F5C9
:105BB0008062904218D002F58062904216D002F5C1
:105BC0008062904214D002F5806290423FF44EAF62
:105BD0000A224EE701224CE702224AE7032248E765
:105BE000042246E7052244E7062242E7072240E76F
:105BF00008223EE702B070BD704700BF0038014088
:105C0000003C014000380240000002400369194294
:105C100001D001207047002070470AB181617047B0
:105C2000090481617047436901EA030221EA030123
:105C300041EA02418161704710B582B01B4B1A6C7A
:105C400042F080521A641B6C03F080530193019B55
:105C5000174A136843F48033136000F0DFF80446FA
:105C6000134B5B6813F4803F08D100F0D7F8001B9A
:105C7000B0F57A7FF4D9032002B010BD0C4A136846
:105C800043F40033136000F0C9F80446084B5B6826
:105C900013F4003F07D100F0C1F8001BB0F57A7F84
:105CA000F4D90320E8E70020E6E700BF003802400F
:105CB00000700040002804DB0901C9B2044B1954EC
:105CC000704700F00F000901C9B2024B1954704728
:105CD00000E400E014ED00E000B500F00700C0F1C2
:105CE000070CBCF1040F28BF4FF0040C031D062B5A
:105CF0000FD9C31E4FF0FF3E0EFA0CF021EA00014F
:105D000099400EFA03FE22EA0E0241EA02005DF813
:105D100004FB0023EEE700000649CB6823F4E063B0
:105D20001B041B0C000200F4E0600343024A1A4308
:105D3000CA60704700ED00E00000FA0510B50446A7
:105D4000054BD868C0F30220FFF7C6FF0146204686
:105D5000FFF7B0FF10BD00BF00ED00E0002807DB3B
:105D600000F01F02400901239340024A42F820300C
:105D7000704700BF00E100E00138B0F1807F0BD236
:105D80004FF0E0235861054AF02182F823100020EB
:105D9000986107221A6170470120704700ED00E00A
:105DA00010B504460E4B1A784FF47A73B3FBF2F336
:105DB0000C4A1068B0FBF3F0FFF7DEFF68B90F2C58
:105DC00001D901200AE0002221464FF0FF30FFF701
:105DD000B5FF054B1C60002000E0012010BD00BF96
:105DE00051000020580000205400002008B5032076
:105DF000FFF792FF0020FFF7D3FFFEF757FA0020CE
:105E000008BD0000034A1168034B1B780B44136064
:105E1000704700BF0806002051000020014B1868A1
:105E2000704700BF0806002038B50446FFF7F6FFAC
:105E30000546B4F1FF3F02D0044B1B781C44FFF72A
:105E4000EDFF401BA042FAD338BD00BF5100002037
:105E5000034B9B68C3F30313024AD35CD8407047DB
:105E60000038024004AD0008034B9B68C3F3822353
:105E7000024AD35CD840704700380240FCAC0008AE
:105E8000034B9B68C3F34233024AD35CD84070474C
:105E900000380240FCAC00080D4B5B6803F4800343
:105EA0009BB90C480A4B5A6802F03F02B0FBF2F073
:105EB0005A68C2F3881202FB00F05B68C3F3014327
:105EC00001335B00B0FBF3F070470348EAE700BF23
:105ED000003802400024F40040787D0108B5074BEB
:105EE0009B6803F00C03042B04D0082B04D1FFF7AC
:105EF000D3FF08BD0248FCE70248FAE70038024039
:105F000040787D010024F40008B5032808D00C284F
:105F10002ED0B0F5406F53D030287AD0002008BD85
:105F2000514BD3F89030034043EA00434F4A934229
:105F300008D0B3F1031F0CD0013A934211D1FFF7FF
:105F4000CDFFECE7484B186810F00200E7D0484856
:105F5000E5E7454B186F10F00200E0D04FF4004029
:105F6000DDE7FFF7BBFFFFF773FFFFF789FFD6E71A
:105F70003D4BD3F89030034043EA00433D4A9342FF
:105F800008D0B3F10C1F0CD0043A934211D1FFF7A3
:105F9000A5FFC4E7344B186810F00200BFD03448A6
:105FA000BDE7314B186F10F00200B8D04FF400403D
:105FB000B5E7FFF793FFFFF74BFFFFF755FFAEE79E
:105FC000294BD3F89030034043EA00432A4A9342D6
:105FD00009D0B3F10C2F0DD0A2F58062934211D1FC
:105FE000FFF77CFF9BE7204B186810F0020096D06B
:105FF0001F4894E71C4B186F10F002008FD04FF42D
:1060000000408CE7FFF76AFFFFF722FFFFF738FF3A
:1060100085E7154BD3F89030034043EA0043174A15
:10602000934208D0B3F1301F0DD0103A934213D1F0
:10603000FFF754FF73E70C4B186810F002003FF4B1
:106040006EAF0B486BE7084B186F10F002003FF47F
:1060500066AF4FF4004062E7FFF740FFFFF7F8FE3E
:10606000FFF702FF5BE700BF0038024002000300B9
:106070000024F40008000C000008000C2000300090
:1060800008B5C0280AD0B0F5407F2FD0B0F5405FEA
:1060900055D0B0F5404F7BD0002008BD524BD3F80F
:1060A0009030034043EA0043504A934208D0B3F192
:1060B000C01F0CD0403A934211D1FFF70FFFECE71D
:1060C000494B186810F00200E7D04948E5E7464B15
:1060D000186F10F00200E0D04FF40040DDE7FFF74A
:1060E000FDFEFFF7B5FEFFF7BFFED6E73E4BD3F848
:1060F0009030034043EA00433E4A934209D0B3F153
:10610000032F0DD0A2F58072934211D1FFF7E6FE66
:10611000C3E7354B186810F00200BED03448BCE726
:10612000314B186F10F00200B7D04FF40040B4E7C5
:10613000FFF7D4FEFFF78CFEFFF796FEADE72A4B84
:10614000D3F89030034043EA00432B4A934209D0EE
:10615000B3F1302F0DD0A2F58052934211D1FFF749
:10616000BDFE9AE7204B186810F0020095D0204839
:1061700093E71D4B186F10F002008ED04FF40040D3
:106180008BE7FFF7ABFEFFF763FEFFF76DFE84E7DB
:10619000154BD3F89030034043EA0043174A93422B
:1061A00009D0B3F1C02F0ED0A2F58042934213D193
:1061B000FFF794FE71E70C4B186810F002003FF4F3
:1061C0006CAF0B4869E7084B186F10F002003FF402
:1061D00064AF4FF4004060E7FFF780FEFFF738FE42
:1061E000FFF742FE59E700BF003802408000C000C0
:1061F0000024F4000002000300200030008000C0F2
:1062000000B5836891FAA1FCBCFA8CFC4FEA4C0CF7
:106210004FF0030E0EFA0CFC23EA0C0391FAA1F1E5
:10622000B1FA81F149008A40134383605DF804FBB1
:1062300000B5C36891FAA1FCBCFA8CFC4FEA4C0C87
:106240004FF0030E0EFA0CFC23EA0C0391FAA1F1B5
:10625000B1FA81F149008A401343C3605DF804FB41
:1062600000B5036A91FAA1FCBCFA8CFC4FEA8C0CD5
:106270004FF00F0E0EFA0CFC23EA0C0391FAA1F179
:10628000B1FA81F189008A40134303625DF804FB8F
:1062900000B5436A090A91FAA1FCBCFA8CFC4FEAEA
:1062A0008C0C4FF00F0E0EFA0CFC23EA0C0391FA43
:1062B000A1F1B1FA81F189008A40134343625DF88C
:1062C00004FB00B5036891FAA1FCBCFA8CFC4FEA10
:1062D0004C0C4FF0030E0EFA0CFC23EA0C0391FA5F
:1062E000A1F1B1FA81F149008A40134303605DF8DE
:1062F00004FBF8B507460E460D6895FAA5F5B5FA04
:1063000085F519E0B26821463846FFF779FF326813
:10631000F1687B6823EA020301FB02F213437B600E
:1063200016E0726921463846FFF7B2FF72682146CF
:106330003846FFF7C6FF0135346834FA05F21BD042
:106340000122AA401440F6D07368013B012BD9D931
:10635000326921463846FFF76BFF7368022BE5D19F
:1063600094FAA4F3B3FA83F3072BDAD872692146BF
:106370003846FFF775FFD9E70020F8BD0B4B1B68C7
:106380000B4AA2FB03235B0A41F2883202FB03F3B0
:106390001A46013B3AB1426B12F0800FF8D0C52388
:1063A0008363002070474FF0004070475800002082
:1063B000D34D621084B00DF1040C8CE80E000B4636
:1063C0001343039A1343049A1343059A1343069AFB
:1063D00013434168034A0A4013434360002004B05A
:1063E000704700BF0081FFFFD0F8800070470B6846
:1063F000C0F88030002070470323036000207047FE
:10640000006800F0030070470B6883604B688A687F
:106410001343CA6813430A691343C2686FF30B023C
:106420001343C360002070470069C0B27047143046
:10643000405870470B6843624B6883628B68CA6838
:1064400013430A6913434A691343C26A22F0F702ED
:106450001343C3620020704710B586B00446002382
:1064600001930293039304934FF48063059301A96E
:10647000FFF7CAFF2046FFF781FF06B010BD0000FE
:1064800038B504460D46504B1B685049A1FB031319
:106490005B0A03FB02F21346013A002B5DD0636BEB
:1064A00013F0450FF7D013F4006FF4D1636B13F0C2
:1064B000040F06D1636B13F0010F05D00120A06318
:1064C0004DE00420A0634AE0C523A3632046FFF704
:1064D000ABFFA84201D0012041E000212046FFF798
:1064E000A6FF03463A481840C8B3002B38DB13F028
:1064F000804F38D113F0005F37D113F0805F36D171
:1065000013F0006F36D113F0806F36D113F0807F17
:1065100036D113F4000F36D113F4800F36D113F4B3
:10652000001F36D113F4801F36D113F4802F36D1DB
:1065300013F4003F36D113F4803F36D113F4004FEB
:1065400036D113F4804F36D113F4005F36D113F0F7
:10655000080F36D04FF4000001E04FF0004038BD86
:106560004FF00070FBE74020F9E78020F7E74FF499
:106570008070F4E74FF40070F1E74FF48060EEE7CD
:106580004FF40060EBE74FF48050E8E74FF4005021
:10659000E5E74FF48040E2E74FF40040DFE74FF4D7
:1065A0000030DCE74FF48020D9E74FF40020D6E735
:1065B0004FF48010D3E74FF40010D0E74FF4800081
:1065C000CDE74FF48030CAE758000020D34D621069
:1065D00008E0FFFD30B587B0044601911025029513
:1065E00040230393002304934FF48063059301A990
:1065F000FFF70AFF41F2883229462046FFF740FFA5
:1066000007B030BD30B587B0044601911125029521
:1066100040230393002304934FF48063059301A95F
:10662000FFF7F2FE41F2883229462046FFF728FFA5
:1066300007B030BD30B587B00446019112250295F0
:1066400040230393002304934FF48063059301A92F
:10665000FFF7DAFE41F2883229462046FFF710FFA5
:1066600007B030BD30B587B00446019118250295BA
:1066700040230393002304934FF48063059301A9FF
:10668000FFF7C2FE41F2883229462046FFF7F8FEA6
:1066900007B030BD30B587B0044601911925029589
:1066A00040230393002304934FF48063059301A9CF
:1066B000FFF7AAFE41F2883229462046FFF7E0FEA6
:1066C00007B030BD30B587B00446002301930C25D8
:1066D00002954022039204934FF48063059301A92D
:1066E000FFF792FE034A29462046FFF7C9FE07B08E
:1066F00030BD00BF00E1F50530B587B0044601921A
:106700000725029540230393002304934FF48063ED
:10671000059301A9FFF778FE41F288322946204609
:10672000FFF7AEFE07B030BD30B587B0044601912B
:106730003725029540230393002304934FF480638D
:10674000059301A9FFF760FE41F2883229462046F1
:10675000FFF796FE07B030BD30B587B00446019113
:106760000625029540230393002304934FF480638E
:10677000059301A9FFF748FE41F2883229462046D9
:10678000FFF77EFE07B030BD30B587B0044600236A
:106790000193332502954022039204934FF48063C2
:1067A000059301A9FFF730FE41F2883229462046C1
:1067B000FFF766FE07B030BD30B587B004460191E3
:1067C0000D25029540230393002304934FF4806327
:1067D000059301A9FFF718FE41F2883229462046A9
:1067E000FFF74EFE07B030BD0146144B1B68144A3C
:1067F000A2FB03235B0A41F2883202FB03F31A4631
:10680000013BBAB14A6B12F0450FF8D012F4006F99
:10681000F5D14B6B13F0040F06D1486B10F001005B
:1068200005D1C5238B63704704208863704701201E
:10683000886370474FF00040704700BF5800002049
:10684000D34D621010B586B0044600230193022296
:106850000292C022039204934FF48063059301A92E
:10686000FFF7D2FD2046FFF7BFFF06B010BD10B501
:1068700086B00446019109230293C02303930023A9
:1068800004934FF48063059301A9FFF7BDFD2046F3
:10689000FFF7AAFF06B010BD0146104B1B68104A57
:1068A000A2FB03235B0A41F2883202FB03F31A4680
:1068B000013B82B14A6B12F0450FF8D012F4006F21
:1068C000F5D1486B10F0040002D1C5238B637047EB
:1068D0000420886370474FF0004070475800002044
:1068E000D34D621010B586B004460A4B0B4301939A
:1068F0002923029340230393002304934FF48063DE
:10690000059301A9FFF780FD2046FFF7C5FF06B0FC
:1069100010BD00BF00001080F8B505460E461746B2
:10692000234B1B68234AA2FB03235B0A41F28832F4
:1069300002FB03F31A46013B8AB36C6B14F0450F5C
:10694000F8D014F4006FF5D16B6B13F0040F06D17F
:106950006B6B13F0010F05D00120A86321E0042028
:10696000A8631EE02846FFF75FFDB04201D001207A
:1069700017E0C523AB6300212846FFF758FD034607
:1069800010F4604008D013F4804F0BD113F4004F83
:106990000BD04FF4805004E01B0C3B8001E04FF023
:1069A0000040F8BD4FF40050FBE74FF48030F8E7AB
:1069B00058000020D34D621070B586B004460D46D5
:1069C00000230193032602964022039204934FF47E
:1069D0008063059301A9FFF717FD2A46314620463B
:1069E000FFF79AFF06B070BD0146164B1B68164AAA
:1069F000A2FB03235B0A41F2883202FB03F31A462F
:106A0000013BE2B14A6B12F0450FF8D012F4006F6F
:106A1000F5D14B6B13F0040F0BD14B6B13F001034B
:106A20000AD1486B10F040000BD040228A63184610
:106A300070470420886370470120886370474FF0D7
:106A40000040704758000020D34D621010B586B04A
:106A500004464FF4D5730193082302934023039314
:106A6000002304934FF48063059301A9FFF7CCFC46
:106A70002046FFF7B9FF06B010BD000070B582B028
:106A80000446002301930068FFF7E6FC054610B1B9
:106A9000284602B070BD2068FFF7D8FF38B901233F
:106AA000A364A36C012B0BD02E46284614E00023D0
:106AB000A3642068FFF7D0FC0028F2D00546E7E782
:106AC00000212068FFF730FE0028EDD04FF0805500
:106AD000DEE7019B01330193019A4FF6FE739A4260
:106AE00013D896B900212068FFF71EFEE0B91249BD
:106AF0002068FFF7F7FE0646C0B900212068FFF7BF
:106B000096FCC30FE5D01E46E3E7019A4FF6FE73ED
:106B10009A420ED810F0804302D001236364B7E795
:106B2000002262641D46B3E70546B1E74FF0805589
:106B3000AEE74FF08075ABE7000010C1F0B589B04B
:106B400004460F46FFF76AF90646002300930193B7
:106B500008212068FFF73EFD054610B1284609B020
:106B6000F0BD216D09042068FFF7DEFD0546002811
:106B7000F4D14FF0FF33029308230393302304939F
:106B800002230593002306930123079302A920689B
:106B9000FFF750FC2068FFF7F7FD054658B1DDE729
:106BA000FFF722FC4DF825000135FFF737F9831B6D
:106BB000B3F1FF3F3FD02068436B13F02A0F07D19A
:106BC000436B13F4001FEBD1436B13F4005FECD164
:106BD000436B13F0080F25D1436B13F0020F24D140
:106BE000456B15F0200523D140F23A538363019A97
:106BF000130203F47F0343EA0263110A01F47F41A5
:106C00000B4343EA12633B60009A130203F47F03D1
:106C100043EA0263110A01F47F410B4343EA126322
:106C20007B609BE70825856398E70225856395E7E8
:106C30002025856392E74FF000458FE710B582B0BD
:106C400004460021009101910068FFF7F0FB10F06D
:106C5000007F13D169462046FFF770FF80B9019B82
:106C600013F4802F0ED0216D09042068FFF75CFD1E
:106C700030B902212068FFF76FFD01E04FF400609A
:106C800002B010BD4FF08060FAE710B582B0044644
:106C90000021009101910068FFF7C9FB10F0007F0F
:106CA00013D169462046FFF749FF80B9019B13F4D1
:106CB000803F0ED0216D09042068FFF735FD30B903
:106CC00000212068FFF748FD01E04FF4006002B0AA
:106CD00010BD4FF08060FAE770B581B104460E46F2
:106CE000016D09040068FFF767FD054608B12846F5
:106CF00070BD00212068FFF79AFB3060F7E74FF086
:106D00000065F4E72DE9F04F87B005460C461646BE
:106D10009B46DDF840A0FFF781F8002C36D0814675
:106D200095F83470FFB2012F40F004810023AB636B
:106D300006EB0B03EA6D93422ED8032385F834301B
:106D40002B680022DA626B6C012B00D076024FF0C8
:106D5000FF3300934FEA4B230193902302930223C6
:106D60000393002304930123059369462868FFF7E2
:106D700061FBBBF1010F14D902232B633146286854
:106D8000FFF758FCA0B9DDF8048038E0AB6B43F0A6
:106D90000063AB630127D2E0AB6B43F00073AB63DE
:106DA000CDE001232B6331462868FFF72BFCE9E790
:106DB0002B68654A9A63AB6B0343AB63012385F889
:106DC000343000232B63BAE02868FFF70DFB2070F6
:106DD000C0F307236370C0F30743A370000EE07095
:106DE0000434A8F104080136072EEDD9FFF716F890
:106DF000A0EB090050450FD2BAF1000F0CD0286863
:106E0000466B16F4957615D1436B13F4004FEDD015
:106E1000B8F1000FEAD0E7E72B684B4A9A63AB6BF7
:106E200043F00043AB63012385F8343000232B6328
:106E3000032784E0436B13F4807F05D0BBF1010F7F
:106E400002D96B6C032B38D12B685A6B12F0080FE8
:106E500044D15A6B12F0020F4CD15A6B12F0200F32
:106E600054D12868436B13F4001F5BD0B8F1000FB6
:106E700058D0FFF7B9FA2070C0F307236370C0F34E
:106E80000743A370000EE0700434A8F10408FEF775
:106E9000C5FFA0EB0900504502D2BAF1000FE0D1C6
:106EA0002B68294A9A63AB6B43F00043AB63012321
:106EB00085F8343000232B6341E0FFF703FC0346E1
:106EC0000028C1D02A6820499163AA6B1343AB63A1
:106ED000012385F8343000232B6330E01A4A9A638B
:106EE000AB6B43F00803AB63012385F83430002318
:106EF0002B6324E0144A9A63AB6B43F00203AB6349
:106F0000012385F8343000232B6318E00E4A9A637E
:106F1000AB6B43F02003AB63012385F834300023CF
:106F20002B630CE040F23A538363012385F834303D
:106F3000002704E0AB6B43F00053AB6301273846F6
:106F400007B0BDE8F08F00BFFF0540002DE9F04F0E
:106F50008BB005460C4616469B46DDF850A0FEF762
:106F60005DFF002C37D0804695F83470FFB2012FBA
:106F700040F0E1800023AB6306EB0B03EA6D934224
:106F80002FD8032385F834302B680022DA626B6C2B
:106F9000012B00D076024FF0FF3304934FEA4B23CE
:106FA00005939023069300230793089301230993E5
:106FB00004A92868FFF73EFABBF1010F16D9202378
:106FC0002B6331462868FFF765FB0190019BABB945
:106FD000DDF8149040E0AB6B43F00063AB63012736
:106FE000AEE0AB6B43F00073AB63A9E010232B63FF
:106FF00031462868FFF736FB0190E7E72B68524AD5
:107000009A63AB6B019A1343AB63012385F8343069
:1070100000232B6394E023780393627843EA0223EE
:107020000393A27843EA02430393E27843EA0263BC
:1070300003930434A9F1040903A92868FFF7D7F9D9
:107040000136072EE7D9FEF7E9FEA0EB0800504510
:107050000FD2BAF1000F0CD02868466B16F48D766B
:1070600015D1436B13F4804FEDD0B9F1000FEAD086
:10707000E7E72B68344A9A63AB6B019A1343AB631F
:10708000012385F8343000232B63032758E0436B3A
:1070900013F4807F05D0BBF1010F02D96B6C032B79
:1070A00018D12B685A6B12F0080F24D15A6B12F0CA
:1070B000020F2CD15A6B12F0100F34D0224A9A636F
:1070C000AB6B43F01003AB63012385F8343000232E
:1070D0002B6335E0FFF7F6FA03460028E1D02A6873
:1070E00019499163AA6B1343AB63012385F83430CC
:1070F00000232B6324E0144A9A63AB6B43F008032C
:10710000AB63012385F8343000232B6318E00E4A6B
:107110009A63AB6B43F00203AB63012385F8343011
:1071200000232B630CE040F23A529A63012385F866
:107130003430002704E0AB6B43F00053AB6301270E
:1071400038460BB0BDE8F08FFF0540000346426EA5
:10715000920F0A70426EC2F383624A7090F8672001
:1071600002F003028A7090F86620CA7090F86520D9
:107170000A7190F864204A71826E120DCA80B0F8CC
:107180006A2002F00F020A72826EC2F3C0324A72A3
:10719000826EC2F380328A72826EC2F34032CA7249
:1071A000826EC2F300320A7300224A73426C002AD4
:1071B00040F08680806E40F6FC7202EA8002D86E53
:1071C00042EA90720A61DA6EC2F3C2620A7593F8FB
:1071D0006F2002F007024A75DA6EC2F342528A75D6
:1071E000DA6EC2F38242CA75DA6EC2F3C2320A762E
:1071F0000A6901325A65087E00F0070002308240B9
:107200005A6591F808C00CF00F0C012000FA0CF040
:107210009865400A00FB02F2DA654FF400721A66C4
:10722000DA6EC2F380324A76DA6EC2F3C6128A761A
:10723000DA6E02F07F02CA761A6FD20F0A771A6FDF
:10724000C2F341724A771A6FC2F382628A771A6F69
:10725000C2F38352CA771A6FC2F3405281F82020DA
:10726000002081F82100B3F8722002F0010281F8B9
:1072700022201A6FC2F3C03281F823201A6FC2F3A2
:10728000803281F824201A6FC2F3403281F8252021
:107290001A6FC2F3003281F826201A6FC2F38122DE
:1072A00081F827201A6FC2F3012281F828201B6F72
:1072B000C3F3460381F82930012381F82A3070474F
:1072C000012A11D1826E120402F47C12B0F86E0011
:1072D00002430A610A69013292025A65DA654FF483
:1072E00000729A651A669BE7026805499163826B92
:1072F00042F080528263012083F83400704700BF5F
:10730000FF05400070B590B004460123ADF812307F
:107310000068FFF775F800286CD0636C032B45D12B
:10732000636C032B5DD1636C032B1DD0BDF8121071
:10733000216509042068FFF79AFA054600285BD109
:1073400000212068FFF773F8606604212068FFF7CA
:107350006EF8A06608212068FFF769F8E0660C2146
:107360002068FFF764F8206704212068FFF75FF8C2
:10737000000DE06405A92046FFF7E8FE00283ED195
:10738000226D120400232068FFF7B6F9054698BB6A
:10739000234653F8106B93E807008DE80700043488
:1073A00094E80E003046FFF705F825E02068FFF767
:1073B00049FA054600BB00212068FFF738F86067EE
:1073C00004212068FFF733F8A06708212068FFF741
:1073D0002EF8E0670C212068FFF729F8C4F8800038
:1073E0009EE70DF112012068FFF7E6FA0546002836
:1073F00099D001E04FF08065284610B070BD4FF085
:107400008055F9E730B58BB004460023049305930B
:10741000069307930893762309930AAB13E90700B1
:107420008DE8070004AB0ECB2068FEF7C3FF18B150
:10743000012528460BB030BD05462268536823F469
:10744000807353602068FEF7D7FF2268536843F4C7
:10745000807353600220FEF7E7FC2046FFF70EFB27
:1074600030B1012584F83450A36B0343A363E0E7F4
:107470002046FFF747FF30B1012584F83450A36B55
:107480000343A363D5E74FF400712068FFF7A2F828
:107490000028CED0236804499963A36B0343A363F8
:1074A000012584F83450C4E7FF054000A8B110B5A9
:1074B000044690F8343063B1032384F83430204616
:1074C000FFF7A0FF58B9A0632063012384F834308C
:1074D00010BD0377FCF78AFFEEE70120704701201B
:1074E000F6E7436C0B60836C4B60C36C8B60036D81
:1074F000CB60436D0B61836D4B61C36D8B61036E1C
:10750000CB6100207047000030B58BB004460D46BB
:10751000032380F83430436C032B1CD0B1F5805F1B
:1075200008D0B1F5006F0AD079B1836B43F00063E6
:10753000836314E0836B43F0805383630FE0FFF7B2
:107540007DFBA36B0343A36309E0FFF79EFBA36BE3
:107550000343A36303E0836B43F080538363A36B14
:10756000C3B12368174A9A63012584F834504FF455
:1075700000712068FFF72EF830B123681149996334
:10758000A36B0343A3630125012384F83430284609
:107590000BB030BD63680493A3680593E36806935A
:1075A000079563690893A36909930AAB13E9070078
:1075B0008DE8070004AB0ECB2068FEF7FBFE00252C
:1075C000D5E700BFFF05400010B582B00446002398
:1075D000019301A9FFF780FB10B1A36B0343A363E1
:1075E0000198C0F3432002B010BD000003460268BA
:1075F00012F0400F36D110B402681D4810400A68DE
:107600004C682243CC6822430C6922434C692243D4
:107610008C692243CC6922430C6A224310431860D0
:107620005868144A02408868B1F816C040EA0C0055
:1076300002435A608A68B2F5006F03D25A6842F476
:1076400080525A600A6AB2F5005F07D00020DA69FA
:1076500022F40062DA615DF8044B70478A8C1A618B
:107660000020F4E70120DA6922F40062DA61704751
:107670004000FFFFFBF0FFFF70B4046A036A23F0D1
:107680000103036242688569124B2B400D681D435C
:1076900024F002048B6823430F4C104EB04218BFF5
:1076A000A0420CBF0124002405D123F00803CE68BA
:1076B0001E4326F004032CB122F440724C6914439B
:1076C0008A692243426085614A684263036270BCF2
:1076D000704700BF8CFFFEFF000001400004014026
:1076E00070B4036A026A22F4807202624268C56959
:1076F000144C2C400E68264323F400738C6843EA34
:107700000423114C114DA84218BFA0420CBF012404
:10771000002406D123F40063CD6843EA052323F453
:1077200080633CB122F440524C6942EA04128C69F5
:1077300042EA04124260C6614A68C263036270BCD6
:10774000704700BF8CFFFEFF0000014000040140B5
:1077500070B4036A026A22F4805202624468C56906
:107760000D4A2A400D6842EA052223F400538D6831
:1077700043EA0533094E0A4DA84218BFB04204D16E
:1077800024F480444D6944EA85144460C2614A6827
:107790000264036270BC7047FF8CFFFE0000014072
:1077A0000004014070B4036A026A22F4803202626B
:1077B0004468426D0D4D15400A682A4323F4003396
:1077C0008D6843EA05430A4E0A4DA84218BFB042ED
:1077D00004D124F480344D6944EA052444604265B0
:1077E0004A688265036270BC704700BF8FFFFEFF6E
:1077F000000001400004014070B4036A026A22F4F0
:10780000801202624468456D0D4A2A400D6842EAC2
:10781000052223F400138D6843EA0553094E0A4DEF
:10782000A84218BFB04204D124F480244D6944EA30
:107830008524446042654A68C265036270BC704733
:10784000FF8FFFFE000001400004014010B4036AF6
:10785000046A24F001040462846924F0F00C4CEA08
:10786000021223F00A030B43826103625DF8044BAA
:10787000704710B4036A046A24F010040462846937
:1078800024F4704C4CEA023223F0A00343EA0113C3
:10789000826103625DF8044B7047836823F07003D4
:1078A0000B4343F00703836070470368196A41F292
:1078B0001112114208D1196A40F24442114203D117
:1078C0001A6822F001021A60012380F83D3000207E
:1078D0007047000090F83D30DBB2012B3AD1022313
:1078E00080F83D300268D36843F00103D360036839
:1078F0001A4AB3F1804F18BF93421DD0A2F57C42C3
:10790000934219D002F58062934215D002F580624D
:10791000934211D002F5784293420DD002F5705295
:10792000934209D0A2F59432934205D01A6842F0EE
:1079300001021A60002070479968094A0A40062A25
:1079400018BFB2F5803F07D01A6842F001021A60F2
:107950000020704701207047002070470000014060
:10796000070001000268D36823F00103D3600368B5
:10797000196A41F21112114208D1196A40F24442C7
:10798000114203D11A6822F001021A60012380F823
:107990003D30002070477047704770477047704710
:1079A000704770B504460368DE681D6915F0020F64
:1079B00010D016F0020F0DD06FF002021A610123F1
:1079C000037703689B6913F0030F64D0FFF7E6FFAA
:1079D0000023237715F0040F12D016F0040F0FD0F8
:1079E00023686FF004021A610223237723689B69DE
:1079F00013F4407F55D02046FFF7D0FF00232377B4
:107A000015F0080F12D016F0080F0FD023686FF092
:107A100008021A61042323772368DB6913F0030F3C
:107A200046D02046FFF7BAFF0023237715F0100F4A
:107A300012D016F0100F0FD023686FF010021A61E9
:107A4000082323772368DB6913F4407F37D020466F
:107A5000FFF7A4FF0023237715F0010F02D016F0E3
:107A6000010F33D115F4025F02D016F0800F35D12B
:107A700015F4807F02D016F0800F37D115F0400F3B
:107A800002D016F0400F39D115F0200F02D016F0B9
:107A9000200F3BD170BDFFF780FF2046FFF77FFF2F
:107AA00096E72046FFF779FF2046FFF778FFA5E726
:107AB0002046FFF772FF2046FFF771FFB4E720462C
:107AC000FFF76BFF2046FFF76AFFC3E723686FF0FD
:107AD00001021A612046FFF75FFFC3E723686FF4D6
:107AE00002521A61204600F0CEFBC1E723686FF412
:107AF00080721A61204600F0C7FBBFE723686FF071
:107B000040021A612046FFF74BFFBDE723686FF084
:107B100020021A61204600F0B5FBBBE730B50368D0
:107B20003F4A904214BF4FF0000E4FF0010EB0F1EB
:107B3000804F14BF72464EF00102AAB9394CA042E0
:107B400014BF00240124384DA8420DD064B904F1BB
:107B5000804404F58234A04214BF0024012405F5BA
:107B60000065A84200D01CB123F070034C68234389
:107B7000002A33D12B4A904214BF002201222A4C02
:107B8000A0422BD052BB02F1804202F582329042D9
:107B900014BF0022012204F50064A0421ED0EAB9FD
:107BA000224A904214BF0022012204F59A34A042D6
:107BB00014D09AB91E4A904214BF0022012204F543
:107BC0000064A0420AD04AB91A4A904214BF002267
:107BD0000122A4F59634A04200D022B123F4407CC7
:107BE000CB6843EA0C0323F080034A691343036024
:107BF0008A68C2620A6882620F4A904214BF734662
:107C00004EF001030BB10B69036301234361036968
:107C100013F0010F03D0036923F00103036130BDAA
:107C20000000014000080040000400400044014002
:107C300000180040002000400004014060B310B56F
:107C4000044690F83D3013B3022384F83D302146BA
:107C500051F8040BFFF762FF012384F8483084F8E1
:107C60003E3084F83F3084F8403084F8413084F866
:107C7000423084F8433084F8443084F8453084F846
:107C8000463084F8473084F83D30002010BD80F83D
:107C90003C30FCF707FCD7E70120704760B310B514
:107CA000044690F83D3013B3022384F83D3021465A
:107CB00051F8040BFFF732FF012384F8483084F8B1
:107CC0003E3084F83F3084F8403084F8413084F806
:107CD000423084F8433084F8443084F8453084F8E6
:107CE000463084F8473084F83D30002010BD80F8DD
:107CF0003C30FFF750FED7E70120704770B4036AAD
:107D0000026A22F01002026242688569144C2C401B
:107D10000D6844EA052523F020038C6843EA041328
:107D2000104C114EB04218BFA0420CBF01240024D9
:107D300006D123F08003CE6843EA061323F0400304
:107D40003CB122F440624C6942EA84028C6942EA06
:107D50008402426085614A688263036270BC704736
:107D6000FF8CFFFE000001400004014038B590F890
:107D70003C30012B00F0958004460D46012380F82D
:107D80003C30142A00F28880DFE802F00B868686F9
:107D90001F86868634868686488686865D868686A3
:107DA00071000068FFF768FC2268936943F00803DC
:107DB00093612268936923F00403936122689369B5
:107DC00029690B439361002067E00068FFF796FF85
:107DD0002268936943F4006393612268936923F4F2
:107DE0008063936122689369296943EA012393615F
:107DF000002052E00068FFF773FC2268D36943F06B
:107E00000803D3612268D36923F00403D361226895
:107E1000D36929690B43D36100203EE00068FFF776
:107E200097FC2268D36943F40063D3612268D36965
:107E300023F48063D3612268D369296943EA01236B
:107E4000D361002029E00068FFF7ACFC2268536D85
:107E500043F0080353652268536D23F00403536510
:107E60002268536D29690B435365002015E00068B3
:107E7000FFF7C2FC2268536D43F400635365226828
:107E8000536D23F4806353652268536D296943EA77
:107E900001235365002000E00120002384F83C30DA
:107EA00038BD0220FCE710B4846824F47F4C42EA19
:107EB00003220A4342EA0C0282605DF8044B7047D9
:107EC00090F83C30012B76D010B50446012380F8A1
:107ED0003C30022380F83D3002689068374B034005
:107EE00093600B68602B4CD023D8402B54D011D812
:107EF000202B03D00AD80BB1102B05D119462068CE
:107F0000FFF7CBFC002028E0012026E0302BF5D045
:107F1000012022E0502B0AD1CA6849682068FFF787
:107F200095FC50212068FFF7B8FC002015E00120E7
:107F300013E0B3F5805F3AD0B3F5005F14D0702B37
:107F400037D1CB684A6889682068FFF7ACFF2268A0
:107F5000936843F0770393600020012384F83D3059
:107F6000002384F83C3010BDCB684A6889682068DB
:107F7000FFF799FF2268936843F4804393600020E1
:107F8000EBE7CA6849682068FFF773FC6021206846
:107F9000FFF783FC0020E0E7CA6849682068FFF724
:107FA00055FC40212068FFF778FC0020D5E7002031
:107FB000D3E70120D1E70220704700BF8800FEFF11
:107FC00001F01F014FF0010C0CFA01FC036A23EAD7
:107FD0000C030362036A8A40134303627047000084
:107FE00010B5044610293CD8DFE801F0093B3B3BC3
:107FF0001F3B3B3B263B3B3B2D3B3B3B340090F840
:108000003E30DBB2013B18BF0123002B40F08980DA
:10801000102974D8DFE801F02C73737363737373E2
:10802000677373736B7373736F0090F83F30DBB2D9
:10803000013B18BF0123E8E790F84030DBB2013B79
:1080400018BF0123E1E790F84130DBB2013B18BFD4
:108050000123DAE790F84230DBB2013B18BF01237D
:10806000D3E790F84330DBB2013B18BF0123CCE7E4
:10807000022384F83E3001222068FFF7A1FF236825
:108080002A492B4A934218BF8B4203D15A6C42F4BF
:1080900000425A642368254AB3F1804F18BF9342C7
:1080A00031D0A2F57C4293422DD002F580629342FA
:1080B00029D002F58062934225D002F5784293429E
:1080C00021D002F5705293421DD0A2F59432934212
:1080D00019D01A6842F001021A60002022E002233F
:1080E00084F83F30C7E7022384F84030C3E7022317
:1080F00084F84130BFE7022384F84230BBE7022313
:1081000084F84330B7E799680A4A0A40062A18BF3C
:10811000B2F5803F07D01A6842F001021A600020D1
:1081200000E0012010BD0020FCE700BF000001407E
:10813000000401400700010038B504460D46002246
:108140000068FFF73DFF23682449254A934218BF82
:108150008B420DD1196A41F21112114208D1196AEC
:1081600040F24442114203D15A6C22F400425A6454
:108170002368196A41F21112114208D1196A40F2BA
:108180004442114203D11A6822F001021A60102DF4
:108190001FD8DFE805F0091E1E1E0E1E1E1E121E31
:1081A0001E1E161E1E1E1A00012384F83E300020DB
:1081B00038BD012384F83F30F9E7012384F84030CB
:1081C000F5E7012384F84130F1E7012384F84230D8
:1081D000EDE7012384F84330E9E700BF00000140E8
:1081E0000004014090F83C20012A45D070B40346B9
:1081F000012280F83C20022280F83D20026850686D
:1082000094681E4E1E4DAA4218BFB24203D120F4FC
:1082100070004D68284320F070000D6828435060BE
:108220001A681648B2F1804F18BF824217D0A0F5E5
:108230007C40824213D000F5806082420FD000F56E
:10824000806082420BD000F57840824207D000F572
:108250007050824203D0A0F59430824204D124F0C1
:108260008004896821439160012283F83D20002029
:1082700083F83C0070BC704702207047000001404A
:1082800000040140704770477047000030B5036834
:108290003B4A904214BF4FF0000E4FF0010EB0F178
:1082A000804F14BF72464EF00102AAB9354CA0426D
:1082B00014BF00240124344DA8420DD064B904F148
:1082C000804404F58234A04214BF0024012405F543
:1082D0000065A84200D01CB123F070034C68234312
:1082E000002A33D1274A904214BF00220122264C93
:1082F000A0422BD052BB02F1804202F58232904262
:1083000014BF0022012204F50064A0421ED0EAB985
:108310001E4A904214BF0022012204F59A34A04262
:1083200014D09AB91A4A904214BF0022012204F5CF
:108330000064A0420AD04AB9164A904214BF0022F3
:108340000122A4F59634A04200D022B123F4407C4F
:10835000CB684CEA030303608A68C2620A888262BF
:108360000D4A904214BF73464EF001030BB10B69E6
:108370000363436943F001034361002030BD00BF44
:10838000000001400008004000040040004401409B
:10839000001800400020004000040140B2F5004FEA
:1083A00006D001EB5301B1FBF3F189B2C160704714
:1083B0005A0802EB4102B2FBF3F34FF6F0721A4097
:1083C000C3F342031343C3607047000038B503682A
:1083D00013F0010F62D104460D460368314A1A407A
:1083E0004B68C9680B4329690B43A9690B431A43BE
:1083F0000260AB68426822F44052134343606B69E9
:10840000826822F4407213438360274B984216D04F
:10841000264B98421BD0264B98421CD0254B9842A5
:108420001DD0254B98421ED0244B984220D0244B7F
:10843000984222D0234B984224D001202FE00320E1
:10844000FDF762FD60B32B680BBB012027E00C2019
:10845000FDF75AFDF6E73020FDF756FDF2E7C020A4
:10846000FDF70EFEEEE74FF44070FDF709FEE9E779
:108470004FF44060FDF748FDE4E74FF44050FDF74E
:10848000FFFDDFE74FF44040FDF7FAFDDAE7AA69A8
:1084900001462046FFF782FF002000E0012038BDA2
:1084A0000120FCE7F369FFEF0010014000440040A9
:1084B00000480040004C00400050004000140140C3
:1084C00000780040007C0040034AD2F8883043F432
:1084D0007003C2F88830704700ED00E008B501462F
:1084E0000122054801F01EFA044B187008B1012062
:1084F00008BD0020FCE700BF5C1600208C020020B5
:1085000008B501460122002001F00CFA034B187057
:1085100008B1012008BD0020FCE700BF8C0200204C
:10852000F8B504460D461646104901F0ECFE104B16
:10853000187008B1C0B2F8BD022221460D4801F002
:1085400021FA0B4B187008B1C0B2F4E7094F0A4B7F
:1085500032462946384601F01AFC054C2070384650
:1085600001F069FD2070C0B2E5E700BF14060020ED
:108570008C0200202C0600200C0600202DE9F04182
:1085800004460F4690461D46434901F0BCFE434B4E
:108590001870E8B901222146414801F0F3F9064676
:1085A0003E4B187018BB29463D4801F059FD3B4B26
:1085B000187058B36420F8F795FB054622463949F0
:1085C000F7F780FE2846F8F795FB344B18780CE057
:1085D0006420F8F787FB054622463349F7F772FE19
:1085E0002846F8F787FB2D4B1878BDE8F08164200A
:1085F000F8F778FB0546234632462C49F7F762FE2A
:108600002846F8F777FB254B1878EEE7284B4246CB
:108610003946234801F0CFFA0646204B187008BBB4
:1086200055B91F4BDA68234B1A603A705A787A7042
:108630009A78BA70DB78FB70194801F0FCFC0546AB
:10864000164B1870D8B16420F8F74CFB0646234649
:108650002A461949F7F736FE3046F8F74BFB0F4B21
:108660001878C2E76420F8F73DFB054623463246FA
:108670001249F7F727FE2846F8F73CFBEFE764209E
:10868000F8F730FB054622460D49F7F71BFE284652
:10869000F8F730FBE3E700BF140600208C0200204F
:1086A0002C06002010AC000854AB000878AB000882
:1086B0001006002080020020C8AB0008A0AB000814
:1086C000F0AB000810B504460C4901F01CFE0C4B41
:1086D000187008B9C0B210BD0B222146094801F03C
:1086E00051F9074B187008B1C0B2F4E7054801F022
:1086F000A2FC034B1870C0B2EDE700BF14060020C7
:108700008C0200202C06002070B504461A4901F0A6
:10871000FAFD1A4B1870A0B9204601F016FE054666
:10872000164B1870D8B96420F8F7DCFA05462246D3
:108730001349F7F7C7FD2846F8F7DCFA0F4B18780E
:1087400070BD6420F8F7CEFA054622460D49F7F7CA
:10875000B9FD2846F8F7CEFA084B1878F0E7642000
:10876000F8F7C0FA064623462A460749F7F7AAFD56
:108770003046F8F7BFFAE1E7140600208C0200202B
:1087800058AC000838AC00087CAC0008F8B50446CA
:108790000D461646104901F0B6FD104B187008B191
:1087A000C0B2F8BD322221460D4801F0EBF80B4B68
:1087B000187008B1C0B2F4E7094F0A4B3246294697
:1087C000384601F0E4FA054C2070384601F033FCDD
:1087D0002070C0B2E5E700BF140600208C02002024
:1087E0002C0600200C06002008B5044B03EB800289
:1087F000526852680344187A904708BDB826002092
:1088000008B5084B1B5C53B9064B01221A5403EB05
:108810008002526812680344187A904708BD00200D
:10882000FCE700BFB826002038B5044C04EB8005F7
:108830006D68AD680444207AA84738BDB82600208A
:1088400038B5044C04EB80056D68ED680444207A6B
:10885000A84738BDB826002010B5044B03EB8004B0
:10886000646824690344187AA04710BDB826002024
:108870004278007840EA02207047C378827842EA62
:108880000322437843EA0223007840EA032070473A
:108890000170090A417070470170C1F307234370EA
:1088A000C1F307438370090EC1707047944632B11B
:1088B0000A78013102700130BCF1010CF8D1704727
:1088C00001700130013AFBD1704784469CF80000EA
:1088D0000CF1010C0B780131C01A013A01D00028CB
:1088E000F4D07047034600E00133187808B188429D
:1088F000FAD1704710B44FF0000C634602E04FF01D
:10890000010C0133012B15D81A01184CA258002A6A
:10891000F5D00468A242F4D1144A02EB0312546861
:1089200082689442EDD1114A02EB031294684269C5
:108930009442E6D1022B0BD0B1B90C4A02EB0313DF
:108940009B89B3F5807F0DD000205DF8044B704704
:10895000022914BF63464CF001030BB10020F4E779
:108960001220F2E71020F0E71020EEE7902600201A
:10897000002000E00130012804D80301034AD35845
:10898000002BF7D1023818BF012070479026002035
:1089900070B4002300E00133012B13D81A01234CDB
:1089A000A45802689442F6D1204A02EB031254689C
:1089B00082689442EFD11D4A02EB03129468426927
:1089C0009442E8D1022B08D0F9B1184A02EB031205
:1089D00092894ABB4FF480721DE00023012B05D819
:1089E0001A01124CA2580AB10133F7E7022B19D031
:1089F0000E4D1C0105EB031206682E51846854606D
:108A00004069906000209081DEE7084A02EB031283
:108A10009289013292B2054901EB03118A81581CF7
:108A200070BC70470020FBE70020F9E7902600208B
:108A30000138012815D80D4B03EB00139B89B3F5C2
:108A4000807F03D043B1013B9BB200E00023074A83
:108A500002EB0012938133B903010020034AD05086
:108A60007047022070470020704700BF902600200A
:108A7000002303E05DF8044B70470133012B11D84C
:108A80001A0109498A588242F7D110B41A01002408
:108A90008C500133012BEDD81A0103498A588242C8
:108AA000F7D1F3E7704700BF9026002002398369B1
:108AB000023B8B4204D94389C06A01FB0300704723
:108AC000002070470268C36A04339089B1FBF0F15B
:108AD0005289B1FBF2F101E0091A0833186818B1A4
:108AE0008142F9D258680844704770B506460D4671
:108AF00001F11A00FFF7BCFE3378032B00D070BDE4
:108B0000044605F11400FFF7B3FE44EA0040F6E71F
:108B100070B506460C46154691B204F11A00FFF7EF
:108B2000B7FE3378032B00D070BD290C04F114007C
:108B3000FFF7AEFEF8E738B500234B72C36973B395
:108B400005460C460022134606E0BCF1090F0FD083
:108B5000A1184B72013263460A2B0ED803F1010CA7
:108B6000296ACB5C202BF6D0052BEED1E523ECE770
:108B7000A1182E2048720132EAE7224400235372E2
:108B80002B6ADB7A2372286A1C30FFF776FE20609E
:108B9000286A1630FFF771FEE080000CA08038BD17
:108BA0002DE9F84F81468A46D1F8008000F1240B68
:108BB0000B2220215846FFF783FE00252B4608276D
:108BC00029E0013618F806302F2BFAD05C2BF8D0AC
:108BD0004644CAF80060002D44D099F82430E52BB3
:108BE00035D0202C37D8042389F82F30002035E0E9
:108BF00014F0800F27D121461B48FFF773FE78BB86
:108C0000A4F16103DBB2192B01D8203CE4B20BF8CC
:108C10000540013533465E1C18F80340202CD7D997
:108C20005C2C18BF2F2CCDD02E2C18BFAF42DFD814
:108C30002E3C18BF01240B2F08BF44F0010464B977
:108C400008250B27E6E7803C084B1C5DD3E705238E
:108C500089F82430C5E70023C6E70620BDE8F88F71
:108C60000620FBE70620F9E79CAC000814AD0008DD
:108C70000146006808B1024603E04FF0FF3070473C
:108C800001321378202B01D93A2BF9D13A2B01D09C
:108C900000207047034613F8010B3038092898BFAD
:108CA0009A4203D128B901320A6070474FF0FF3071
:108CB00070474FF0FF30704738B50D46044698B105
:108CC00003689BB11A78A2B18188DA88914203D0F7
:108CD000092000242C6038BD5878FFF785FD10F07E
:108CE000010009D12468F5E70920F3E71C460920B3
:108CF000F0E709200024EDE709200024EAE72DE948
:108D0000F041C57815B92846BDE8F0810446076BE7
:108D100000F1340801233A4641464078FFF790FDC0
:108D20000546A0B90023E370636AFB1AE269934227
:108D3000E9D2A67808E0E3691F4401233A46414698
:108D40006078FFF77DFD013E012EF4D8DBE70125B9
:108D5000D9E770B5036B8B4202D10026304670BD57
:108D600004460D46FFF7CBFF06460028F6D1012347
:108D70002A4604F134016078FFF756FD10B1012650
:108D80004FF0FF352563E9E738B504460023C3708B
:108D90004FF0FF330363FFF7DCFF30BB054604F2FF
:108DA0003220FFF765FD4AF6552398421FD194F80B
:108DB0003430E92B07D0636B03F0FF130D4A934265
:108DC00001D0022514E004F16A00FFF756FD20F0FF
:108DD0007F40094B98420BD004F18600FFF74DFD10
:108DE000064B984204D0022502E0042500E003254A
:108DF000284638BDEB0090004641540046415433AC
:108E00002DE9F04F87B00D46164600230B60FFF7A3
:108E10002FFF071EC0F26781BE4B53F82740002C7E
:108E200000F066812C6006F0FE06237873B160784E
:108E3000FFF7DAFC10F0010508D1002E00F0548194
:108E400010F0040F00F050810A254DE1002323703B
:108E5000F8B26070FFF7D4FC10F0010F40F04A81C7
:108E60001EB110F0040F40F0478104F10C02022102
:108E70006078FFF7F1FC0546002840F03F81A289A9
:108E8000A2F500739BB2B3F5606F00F23981531EF7
:108E90001A4201D0012527E100212046FFF774FF87
:108EA000022800F088800026042800F02B81012889
:108EB00000F22A8104F13F00FFF7DAFCB4F80C80DD
:108EC000404540F0238104F14A00FFF7D1FC0746FA
:108ED00020B904F15800FFF7D0FC0746E76194F889
:108EE0004420A270531EDBB2012B00F2118107FB5C
:108EF00002F3009394F84190A4F80A90B9F1000F9E
:108F000000F0108109F1FF3319EA030F40F00C81E2
:108F100004F14500FFF7ACFC824620814FEA581B64
:108F2000B0FBFBF30BFB13039BB2002B40F0FE8066
:108F300004F14700FFF79CFC019020B904F15400B4
:108F4000FFF79BFC019004F14200FFF791FC014602
:108F5000002800F0ED80009BC318BAFBFBFB5B44CC
:108F6000019A9A42C0F0E680D21AB2FBF9F04A4563
:108F7000C0F0E2804FF6F572904234D840F6F572B8
:108F800090426AD94FF0020B2FE0002006AB03EBB2
:108F9000860343F8100C0136032E0ED804F134007A
:108FA000330103F5DF7318440379002BEDD008304B
:108FB000FFF763FCEAE70026EEE700270AE0314608
:108FC0002046FFF7E1FE01287FF66EAF0137032F41
:108FD0003FF66AAF06AB03EB870353F8106C002E25
:108FE000EDD10320F2E74FF0030B00F10209C4F8C2
:108FF000189026628A1962623344E362BBF1030F60
:109000002ED0BAF1000F00F09D80009B1A44A2629E
:10901000BBF1020F35D009EB490209F0010303EB64
:1090200052034344013BB3FBF8F3BB4200F28C8094
:109030004FF0FF336361236180232371BBF1030F82
:1090400022D084F800B0344A138801339BB21380D5
:10905000E3802046FFF70CFD46E04FF0010BC4E72C
:1090600004F15E00FFF704FC002867D1BAF1000F9D
:1090700066D104F16000FFF700FCA0624FEA8903AB
:10908000CFE74FEA4903CCE704F16400FFF7F0FBB8
:109090000128D6D1711C2046FFF75BFE0028D0D1F5
:1090A0000023237104F23220FFF7E2FB4AF6552336
:1090B0009842C6D104F13400FFF7DFFB174B98420A
:1090C000BFD104F50670FFF7D8FB154B9842B8D115
:1090D00004F50770FFF7D1FB606104F50870FFF736
:1090E000CCFB2061ADE70B25284607B0BDE8F08F2B
:1090F0000C25F9E70325F7E70A25F5E70125F3E74E
:109100000125F1E70125EFE70D25EDE70D25EBE75B
:109110000D25E9E7B4260020B02600205252614117
:10912000727241610D25DFE70D25DDE70D25DBE7D7
:109130000D25D9E70D25D7E70D25D5E70D25D3E773
:109140000D25D1E70D25CFE70D25CDE72DE9F0471A
:10915000012940F28E8004460D46174683698B42F2
:1091600040F28B800378022B49D0032B60D0012B77
:1091700040F0858001EB5108416A8389B8FBF3F325
:109180001944FFF7E6FD0646002873D104F1340ABE
:1091900008F10109A389B8FBF3F203FB128815F06B
:1091A000010522D01AF8083003F00F0343EA071331
:1091B000DBB20AF808300123E370616AA389B9FBC6
:1091C000F3F319442046FFF7C4FD0646002851D1A9
:1091D000A389B9FBF3F203FB129945B1C7F3071357
:1091E0000AF809300123E37044E0FBB2E1E71AF822
:1091F0000930C7F3032223F00F031343F0E7416A5A
:1092000083895B08B5FBF3F31944FFF7A2FD06461B
:1092100080BB04F134006D00A389B5FBF3F203FBBE
:109220001255B9B22844FFF733FB0123E37021E064
:10923000416A83899B08B5FBF3F31944FFF789FD65
:109240000646B8B927F0704704F13403AD00A2898F
:10925000B5FBF2F102FB11551D442846FFF70DFB4B
:1092600000F0704139432846FFF716FB0123E370F5
:1092700000E002263046BDE8F0870226FAE7022623
:10928000F8E7F8B5056801296AD90C46AB698B4245
:1092900068D92B78022B35D0032B49D0012B63D111
:1092A00001EB5106696AAB89B6FBF3F31944284612
:1092B000FFF74FFD10B14FF0FF3052E0771CAB8944
:1092C000B6FBF3F203FB12662E4496F83460696A2B
:1092D000B7FBF3F319442846FFF73BFD002845D1BF
:1092E000AB89B7FBF3F203FB12772F4497F83430C6
:1092F00046EA032014F0010F01D0000931E0C0F369
:109300000B002EE0696AAB895B08B4FBF3F31944E8
:109310002846FFF71EFD60BB05F134006400AB89F1
:10932000B4FBF3F203FB12442044FFF7A1FA18E068
:10933000696AAB899B08B4FBF3F319442846FFF72D
:1093400008FDC8B905F13400A400AB89B4FBF3F201
:1093500003FB12442044FFF790FA20F0704000E035
:109360000120F8BD0120FCE70120FAE74FF0FF30B3
:10937000F7E74FF0FF30F4E74FF0FF30F1E72DE96A
:10938000F041D0F80080B1F5001F49D207460E46E3
:1093900011F01F0F47D1416184681CBB98F8003061
:1093A000022B01D9D8F82840E4B9B8F80830B3EB5B
:1093B000561F3AD9D8F82830FB61BC61FB69E3B38A
:1093C000B8F80C20B6FBF2F21344FB6108F1340349
:1093D000B8F80C20B6FBF2F102FB11610B443B62C2
:1093E00000201EE0B8F80A50B8F80C3003FB05F571
:1093F000AE420FD321463846FFF743FF0446B0F193
:10940000FF3F14D0012814D9D8F81830834212D95C
:10941000761BEDE721464046FFF748FBF861CCE7B5
:109420000220BDE8F0810220FBE70220F9E70120DD
:10943000F7E70220F5E70220F3E70220F1E72DE944
:10944000F041054606680F4651B9D6F81080B8F1CC
:10945000000F12D0B369434511D84FF001080EE058
:10946000FFF70FFF034601284CD9B0F1FF3F4ED064
:10947000B26982424BD8B84601E04FF00108444639
:109480000CE021462846FFF7FCFE034678B1B0F118
:10949000FF3F18BF01283AD0444537D00134B369A3
:1094A000A342EED8B8F1010F2ED90224E9E74FF01C
:1094B000FF3221463046FFF749FE0246B0FA80F0FF
:1094C0004009002F08BF002070B9A2B93461726949
:1094D000B369023B9A4201D8013A7261337943F091
:1094E00001033371234612E0224639463046FFF726
:1094F0002DFE0246E9E7012A01D0012307E04FF0E3
:10950000FF3304E0012302E0002300E000231846BB
:10951000BDE8F081F8B50C46056801292ED906464C
:109520001146AB69A3422BD94AB14FF0FF3228460E
:10953000FFF70CFE074610B123E0A24221D92746CF
:1095400021463046FFF79DFE0446E0B101281CD0BD
:10955000B0F1FF3F1BD0002239462846FFF7F6FD49
:10956000074670B96B69AA69911E8B42E5D2013337
:109570006B612B7943F001032B71DEE7022700E0DA
:1095800002273846F8BD0027FBE70227F9E7012745
:10959000F7E738B504460568C1692846FFF7D9FBE7
:1095A00020B9236AE5221A700123EB7038BD2DE93A
:1095B000F84306684469C369002B74D005460F461A
:1095C0002034B4F5001F70D2B189B4FBF1F201FB75
:1095D00012423AB90133C3618169A1B93389B3EB4E
:1095E000541F0CD96C6106F13403B289B4FBF2F15B
:1095F00002FB114423442B620020BDE8F8830023C2
:10960000C3610420F9E7B289B4FBF2F27389013B2C
:1096100012EA0308E6D1FFF734FE8146012846D955
:10962000B0F1FF3F45D0B369834234D88FB1A96907
:109630002846FFF704FF814600283CD001283CD093
:10964000B0F1FF3F3BD03046FFF759FB28B1012076
:10965000D3E70023EB610420CFE7B289002106F1B4
:109660003400FFF72DF949463046FFF71FFA306303
:10967000738998450BD20123F3703046FFF73FFB07
:10968000F8B908F10108336B01333363F0E7336B4A
:10969000A3EB08033363C5F8189049463046FFF73B
:1096A00005FAE8619EE70420A7E70420A5E7022069
:1096B000A3E70120A1E707209FE702209DE7012003
:1096C0009BE7012099E770B5044606680021FFF783
:1096D00056FE054640B1284670BD00212046FFF7E2
:1096E00066FF05460028F6D1E1693046FFF731FBF9
:1096F00005460028EFD1206A03787BB1C37A03F0D6
:109700003F03A371C37A13F0080FE6D10B2204F1D3
:109710002401FFF7DAF80028DFD1DCE70425DAE7D7
:1097200030B583B004460191056801E0013301932F
:10973000019B1A782F2AF9D05C2AF7D00022A26068
:109740001B781F2B21D901A92046FFF729FA0346D0
:1097500018BB2046FFF7B7FF94F82F200346F8B94F
:1097600012F0040F19D1A37913F0100F1FD005F1D7
:1097700034016369AA89B3FBF2F002FB1033194488
:109780002846FFF7B2F9A060DDE7802384F82F3088
:1097900011462046FFF7F3FD0346184603B030BDDF
:1097A0000428FAD112F0040FF7D10523F5E70523B9
:1097B000F3E7F8B504460E4607680021FFF7DFFD22
:1097C0000246B8B9002506E0002501212046FFF732
:1097D000EEFE024670B9E1693846FFF7BAFA024672
:1097E00040B9236A1B78002B18BFE52BECD101355B
:1097F000B542EAD1042A01D01046F8BD0722FBE7A2
:1098000070B5044606680121FFF7D3FF054608B18D
:10981000284670BDE1693046FFF79BFA05460028EF
:10982000F6D120220021206AFFF74AF80B2204F12A
:109830002401206AFFF73AF80123F370E8E7F8B54E
:1098400004460E460568042705E000212046FFF780
:10985000AEFE0746E8B9E169D9B12846FFF779FAC3
:109860000746B0B9236A1A7892B1DB7A03F03F0356
:10987000A371E52A18BF2E2AE7D00F2BE5D023F0DD
:109880002003082B14BF00230123B342DDD100E0E5
:1098900004270FB10023E3613846F8BD70B50446D4
:1098A000FFF72DFA054648B92378032B08D000228C
:1098B00011466078FEF7D0FF00B10125284670BD43
:1098C0002379012BF3D104F13406A289002130461B
:1098D000FEF7F6FF4AF6552104F23220FEF7D8FFD4
:1098E0000E493046FEF7D8FF0D4904F50670FEF725
:1098F000D3FF616904F50770FEF7CEFF216904F517
:109900000870FEF7C9FF226A013222630123314643
:109910006078FEF795FF00232371C8E7525261413A
:109920007272416170B584B0019000911646039146
:1099300003A8FFF79DF9041E20DB114B53F82450B8
:1099400025B12846FFF794F800232B70019B0BB13B
:1099500000221A70019B0A4A42F82430721E18BF76
:109960000122002B08BF42F0010212B1002004B016
:1099700070BD01A96846FFF743FAF8E70B20F6E748
:10998000B42600202DE9F04391B00191002800F0A9
:1099900010811446064602F03F073A4603A901A883
:1099A000FFF72EFA054628B100233360284611B090
:1099B000BDE8F083039B0493019904A8FFF7B0FE70
:1099C000054660B99DF93F30002B52DB14F03E0F85
:1099D00014BF0121002104A8FEF78CFF054614F0F6
:1099E0001C0F5CD0002D50D0042D44D047F0080748
:1099F000002DD9D117F0080F61D0FAF7D5F9044638
:109A000001460C980E30FEF747FF21460C981630A1
:109A1000FEF742FF0C9B2022DA72DDF80C80DDF8A5
:109A2000309049464046FFF760F804460022494618
:109A30004046FFF76DF800210C981C30FEF72CFF14
:109A4000039B0122DA70002C39D0039BD3F83080BD
:109A50000022214604A8FFF75DFD05460028A3D19A
:109A600041460398FFF775F90546013C039B1C61CD
:109A700025E00625B3E7FEF77BFF08B91225B5E719
:109A800004A8FFF7BDFE0546B0E79DF8163013F0B9
:109A9000110F13D114F0040FAAD0082584E7002D6C
:109AA00082D19DF8163013F0100F7ED114F0020F02
:109AB00005D013F0010F02D0072575E70725002D0B
:109AC0007FF472AF17F0080F01D047F04007039BF7
:109AD0001B6B73620C9BB362012F94BF00210121A9
:109AE00004A8FEF755FF306108B902255CE7039C26
:109AF000DDF8308041462046FEF7F7FFB06008F100
:109B00001C00FEF7BAFEF0600021F1623460E388C9
:109B1000B380377571753162B16106F130084FF469
:109B200080524046FEF7CCFE17F0200F39D0F46883
:109B3000002C36D0B461039B5F899B8903FB07F738
:109B4000B16801E00225E41BBC4294BF002301235D
:109B50005DB953B13046FFF794FB01460128F1D9B6
:109B6000B0F1FF3FEFD10125EDE7F161002D7FF46A
:109B70001BAF039FB7F80C90B4FBF9F309FB134339
:109B80007BB13846FEF792FF08B902250CE7B4FB1B
:109B9000F9F202443262012341467878FEF744FE2E
:109BA00028B9002D3FF402AFFEE60425FCE60125AE
:109BB000FAE60925FAE62DE9F04F85B004460F468E
:109BC000154698460023C8F8003003A9FFF774F83B
:109BD0000190002840F0B980637D0193002B40F094
:109BE000B480237D13F0010F00F0CE80E668A369F6
:109BF000F61AAE4267D32E4665E0E36A1BB12046F3
:109C0000FEF760FF73E0E1692046FFF73AFB6EE084
:109C10004FF0020A84F815A0CDF804A095E04FF0AB
:109C2000010A84F815A0CDF804A08EE04FF0020AD6
:109C300084F815A0CDF804A087E094F91430002B27
:109C400004DB039B9D890AFB05F532E0236AA3EB45
:109C500009035345F5D2039A928904F1300102FBBE
:109C60000370FEF723FEECE7226A4A450DD094F913
:109C70001430002B6DDB01234A4604F130010398B8
:109C80004078FEF7D1FD002877D1C4F82090039BDF
:109C90009D89A369B3FBF5F205FB1233ED1AAE42C1
:109CA00000D2354604F130012A4619443846FEF701
:109CB000FDFD2F44A3692B44A361D8F800302B4449
:109CC000C8F80030761B002E3FD0A169039A958911
:109CD000B1FBF5F305FB1313002BD8D1B1FBF5F560
:109CE0005389013B1D4008D1002986D1A068012875
:109CF0008ED9B0F1FF3F92D0E061DDF80CB0E169A0
:109D00005846FEF7D3FE814600288FD0A944BBF801
:109D10000C30B6FBF3FAB342A6D805EB0A03BBF846
:109D20000A20934201D9A2EB050A53464A46394616
:109D30009BF80100FEF778FD00283FF47EAF4FF05E
:109D4000010A84F815A0CDF804A0019805B0BDE87B
:109D5000F08F012304F130019BF80100FEF770FD44
:109D600020B9237D03F07F03237584E74FF0010AB8
:109D700084F815A0CDF804A0E7E74FF0010A84F8B5
:109D800015A0CDF804A0E0E707230193DDE72DE956
:109D9000F04F85B004460F46154698460023C8F894
:109DA000003003A9FEF788FF019000284AD1637DA7
:109DB0000193002B46D1237D13F0020F00F0EC80BD
:109DC000A369EB42C0F0B680DD43B3E0E36A002B49
:109DD0003CD02046FEF776FE002800F0D88001280F
:109DE00039D0B0F1FF3F3DD0E061A36803B9A06076
:109DF00094F91430002B3CDBDDF80CB0E1695846D7
:109E0000FEF754FE8146002848D0B144BBF80C3020
:109E1000B5FBF3FAAB425FD806EB0A03BBF80A20A6
:109E2000934201D9A2EB060A53464A4639469BF8AB
:109E30000100FEF705FDC0B34FF0010A84F815A03C
:109E4000CDF804A0019805B0BDE8F08FE169204687
:109E5000FFF7F5FAC0E74FF0020A84F815A0CDF835
:109E600004A0EFE74FF0010A84F815A0CDF804A094
:109E7000E8E70123226A04F1300103984078FEF7F5
:109E8000DFFC20B9237D03F07F032375B4E74FF097
:109E9000010A84F815A0CDF804A0D3E74FF0020A18
:109EA00084F815A0CDF804A0CCE7236AA3EB09033E
:109EB000534504D3039B9E890AFB06F62BE0039AC5
:109EC000928902FB037104F13000FEF7EFFC237D61
:109ED00003F07F032375EDE7236A4B4503D0A269A6
:109EE000E3689A4242D3C4F82090039B9E89A369F9
:109EF000B3FBF6F206FB1233F61AB54200D22E4639
:109F000004F13000324639461844FEF7CFFC237D79
:109F100063F07F0323753744A3693344A361E26888
:109F2000934238BF1346E360D8F800303344C8F892
:109F30000030AD1B5DB3A169039A9689B1FBF6F3BE
:109F400006FB1313002BD0D1B1FBF6F65389013B6E
:109F50001E407FF44DAF00297FF438AFA068002881
:109F60007FF43DAF2046FFF76AFA35E701234A4602
:109F700004F130019BF80100FEF756FC0028B2D036
:109F80004FF0010A84F815A0CDF804A05AE7237D0C
:109F900043F04003237555E70723019352E770B55B
:109FA00082B0044601A9FEF787FE70B9237D13F045
:109FB000400F0AD013F0800F09D1F9F7F5FE0546DE
:109FC000616A0198FEF7C5FE78B102B070BD012349
:109FD000226A04F1300101984078FEF731FC40BB61
:109FE000237D03F07F032375E7E7A66AF37A43F046
:109FF0002003F372A26831462068FEF789FDE1680C
:10A0000006F11C00FEF748FC294606F11600FEF793
:10A0100043FC002106F11200FEF73AFC019B0122ED
:10A02000DA700198FFF73AFC237D23F04003237593
:10A03000CBE70120C9E710B582B00446FFF7AFFFB8
:10A0400008B102B010BD01A92046FEF735FE002878
:10A05000F7D12069FEF7ECFC0028F2D12060F0E790
:10A060002DE9F04F83B004460D4601A9FEF724FE0A
:10A07000064678B9667D6EB9E36A002B00F08E80E3
:10A08000B5F1FF3F0AD0E768AF4200D32F46A76182
:10A09000002F3FD1304603B0BDE8F08F984658F806
:10A0A00004BBD4F808A0BAF1000F27D04FF0020982
:10A0B00009F102095146002701370D462046FFF7F6
:10A0C000E0F80146012813D9B0F1FF3F13D0013564
:10A0D0008542F1D0CB4505D3434643F8087BC8F809
:10A0E00004A09846019B9B698B4209D98A46DFE709
:10A0F00002266675CEE701266675CBE74FF00209AA
:10A10000E36AC3F80090D94500F2FB800023C8F849
:10A110000030BFE77D1E29462046FEF7D3FC0146EE
:10A12000E061DDF804804046FEF7C0FC00B3B8F8FB
:10A130000C30B5FBF3F5B8F80A20013A1540054498
:10A14000B7FBF3F203FB1277002FA3D0226AAA42D7
:10A15000A0D094F91430002B0DDB01232A4604F122
:10A16000300101984078FEF75FFBA0B9256291E7C6
:10A17000022666758EE7012304F1300198F801008C
:10A18000FEF75EFB20B9237D03F07F032375E4E730
:10A19000012666757EE7012666757BE7E368AB42BC
:10A1A00004D2227D12F0020F00D11D46A3690022C5
:10A1B000A261E5B1019AB2F80A80928902FB08F81F
:10A1C00073B16A1EB2FBF8F2013BB3FBF8F18A42AD
:10A1D00006D3C8F100021340A361EF1AE56904E059
:10A1E000A06850B3E0612F460546002D45D1A36914
:10A1F000E268934204D9E360227D42F04002227576
:10A2000001988289B3FBF2F102FB1133002B3FF47A
:10A2100041AF226AAA423FF43DAF94F91430002BBB
:10A220005DDB01232A4604F1300101984078FEF7F6
:10A23000FBFA002862D125622CE700212046FFF7B7
:10A24000FEF8012804D0B0F1FF3F04D0A060C9E7B8
:10A25000022666751EE7012666751BE7294620461D
:10A26000FFF70FF80546B5F1FF3F2DD0012D2ED990
:10A27000019B9B69AB422AD9E561474510D9A7EB01
:10A280000807A3694344A361237D13F0020FE5D0BF
:10A2900029462046FFF7D3F805460028E3D10746B4
:10A2A000A3693B44A3610198B0F80C80B7FBF8F3B5
:10A2B00008FB13738BB12946FEF7F8FB054648B13E
:10A2C000B7FBF8F73D4492E701266675E2E6022601
:10A2D0006675DFE602266675DCE61D4687E7012324
:10A2E00004F130014078FEF7ABFA20B9237D03F08A
:10A2F0007F03237595E701266675CBE60126667513
:10A30000C8E61126C6E630B58FB001900C46002293
:10A3100002A901A8FEF774FD054610B128460FB04A
:10A3200030BD019902A8FFF7FBF905460028F5D1D9
:10A330009DF93730002B06DB002CEFD0214602A818
:10A34000FEF7F9FBEAE70625E8E7F0B59DB00190D6
:10A35000022203A901A8FEF753FD039B10930446B4
:10A3600010B120461DB0F0BD019910A8FFF7D8F933
:10A3700004460028F5D1022110A8FEF7BBFA0446D6
:10A380000028EED19DF96F30002B3CDB9DF8465044
:10A3900015F0010F39D1039F18993846FEF7A5FB38
:10A3A000064615F0100F13D1002CDAD110A8FFF7D4
:10A3B000F0F80446B0FA80F04009002E08BF0020F3
:10A3C000D0B9002CCDD10398FFF768FA0446C8E74E
:10A3D00004970690002104A8FEF7D1FF0446002848
:10A3E000BFD1002104A8FFF72AFA044610B10428BF
:10A3F000DAD1DBE70724D7E70022314610A8FFF7C0
:10A4000089F80446DDE70624ABE70724A9E7000046
:10A41000134B5B7A13BB10B5044603F0FF00104BDF
:10A4200093F809C05FFA8CFC4FF0000E03F80CE0C3
:10A4300093F809C003EB8C0CCCF804405C7A1C4404
:10A4400022725A7A541CE4B25C7230320A703A2397
:10A450004B702F238B7081F803E010BD01207047F3
:10A46000B826002008B50022FFF7D2FF08BD000083
:10A4700010B503460C4A0D490D48006840B10C4820
:10A4800000680344521A934206D8094A136010BD6B
:10A490000748084C0460F2E7F6F7B0F90C230360B4
:10A4A0004FF0FF30F3E700BF00000820004000003D
:10A4B000C4260020C8260020026852E8003F23F48A
:10A4C000907342E800310029F6D1026802F10803D6
:10A4D00053E8003F23F00103083242E8003100292D
:10A4E000F3D1036E012B06D02023C0F88030002367
:10A4F000036683667047026852E8003F23F010034A
:10A5000042E800310029F6D1EEE7000010B504461C
:10A5100083680269134342691343C26913430168A4
:10A520000868914A02401A430A602268536823F47B
:10A530004053E1680B435360A269236A1A432168C0
:10A540008B6823F4306313438B602368874A9342FC
:10A5500018D0874A93423AD0864A93424FD0864ACF
:10A5600093425ED0854A93426DD0854A93427FD014
:10A57000844A934200F09180834A934200F0A28083
:10A5800010230BE0814BD3F8903003F00303032B2F
:10A590001BD8DFE803F00216AB180123E069B0F521
:10A5A000004F00F0D780082B00F23881DFE813F06D
:10A5B00014012701120136012A0136013601360144
:10A5C0002D010423EAE70823E8E71023E6E76F4BB1
:10A5D000D3F8903003F00C030C2B0ED8DFE803F017
:10A5E000070D0D0D090D0D0D880D0D0D0B00002330
:10A5F000D4E70423D2E70823D0E71023CEE7634B48
:10A60000D3F8903003F03003202B73D005D8002B03
:10A6100072D0102B72D10423C0E7302B70D10823E5
:10A62000BCE75A4BD3F8903003F0C003802B69D0BD
:10A6300005D8002B68D0402B68D10423AEE7C02B8F
:10A6400066D10823AAE7514BD3F8903003F4407346
:10A65000B3F5007F5ED006D8002B5DD0B3F5807FC8
:10A660005CD104239AE7B3F5407F59D1082395E7DD
:10A67000464BD3F8903003F44063B3F5006F51D0EC
:10A6800006D8002B50D0B3F5806F4FD1042385E757
:10A69000B3F5406F4CD1082380E73C4BD3F89030A2
:10A6A00003F44053B3F5005F44D006D8002B43D0E9
:10A6B000B3F5805F42D1042370E7B3F5405F3FD12B
:10A6C00008236BE7314BD3F8903003F44043B3F5E4
:10A6D000004F37D005D8BBB3B3F5804F36D1042334
:10A6E0005CE7B3F5404F33D1082357E7022355E722
:10A6F000022353E7022351E700234FE710234DE7DE
:10A7000010234BE7022349E7002347E7102345E7DF
:10A71000102343E7022341E700233FE710233DE7EF
:10A7200010233BE7022339E7012337E7102335E7FE
:10A73000102333E7022331E700232FE710232DE70F
:10A7400010232BE7022329E7002327E7102325E71F
:10A75000102323E7082B5BD8DFE803F01A343A5ABA
:10A76000375A5A5A1E0000BFF369FFEF001001402C
:10A770000044004000480040004C004000500040B1
:10A780000014014000780040007C00400038024086
:10A79000FAF71AFE00283DD06268530803EB400325
:10A7A000B3FBF2F3A3F110014FF6EF72914233D8ED
:10A7B0009AB222F00F02C3F3420313432268D3601C
:10A7C000002030E0FAF710FEE4E7FAF7EDFCE1E7ED
:10A7D0001748E1E7164802E0FAF7F6FD00B36368B0
:10A7E00000EB5300B0FBF3F0A0F110024FF6EF7353
:10A7F0009A4217D8236880B2D860002013E0FAF795
:10A80000F3FDEBE7FAF7D0FCE8E74FF40040E6E7AA
:10A81000012008E0002006E0012004E0012002E021
:10A82000002000E001200023A366E36610BD00BF06
:10A830000024F400436A13F0080F06D0026853683E
:10A8400023F40043416B0B435360436A13F0010F41
:10A8500006D00268536823F40033816A0B435360C7
:10A86000436A13F0020F06D00268536823F4803362
:10A87000C16A0B435360436A13F0040F06D00268A9
:10A88000536823F48023016B0B435360436A13F036
:10A89000100F06D00268936823F48053816B0B433A
:10A8A0009360436A13F0200F06D00268936823F484
:10A8B0000053C16B0B439360436A13F0400F0AD0FF
:10A8C0000268536823F48013016C0B435360036CDC
:10A8D000B3F5801F0BD0436A13F0800F06D00268D7
:10A8E000536823F40023816C0B4353607047026864
:10A8F000536823F4C003416C0B435360EBE72DE92D
:10A90000F84305460E4617469946DDF820802B6829
:10A91000DC6936EA04040CBF01240024BC423AD1AD
:10A92000B8F1FF3FF3D0FBF779FAA0EB09004045FF
:10A9300034D8B8F1000F33D02B681A6812F0040F26
:10A94000E5D0B6F1400218BF0122802EDFD0002AE8
:10A95000DDD0DA6912F0080F11D1DA6912F4006F54
:10A96000D5D04FF400621A622846FFF7A5FD2023D8
:10A97000C5F88430002385F8783003200CE00824E3
:10A980001C622846FFF798FDC5F88440002385F82F
:10A990007830012000E00020BDE8F8830320FBE7C9
:10A9A0000320F9E730B583B004460023C0F88430B3
:10A9B000FBF734FA05462268126812F0080F0FD12F
:10A9C00023681B6813F0040F26D12023E367C4F823
:10A9D000803000202066606684F8780003B030BDC7
:10A9E0006FF07E430093034600224FF4001120468F
:10A9F000FFF785FF0028E3D0226852E8003F23F0EC
:10AA0000800342E800310029F6D12023E3670023C8
:10AA100084F878300320E1E76FF07E4300932B4603
:10AA200000224FF480012046FFF769FF0028CCD0B8
:10AA3000226852E8003F23F4907342E80031002975
:10AA4000F6D1226802F1080353E8003F23F0010326
:10AA5000083242E800310029F3D12023C4F88030C5
:10AA6000002384F878300320B8E768B310B50446B3
:10AA7000C36F03B32423E3672268136823F0010341
:10AA80001360636AE3B92046FFF740FD012811D047
:10AA90002268536823F4904353602268936823F03C
:10AAA0002A0393602268136843F001031360204671
:10AAB000FFF778FF10BD80F87830F9F799FDD9E7F6
:10AAC0002046FFF7B7FEDEE701207047DFF834D0FD
:10AAD000FDF7FAFC0C480D490D4A002302E0D4585A
:10AAE000C4500433C4188C42F9D30A4A0A4C0023D8
:10AAF00001E013600432A242FBD3F5F705FEF8F73C
:10AB000017FB704700000820000000205C000020B8
:10AB1000A4AD00085C000020C8260020FEE700006D
:10AB2000F8B500BFF8BC08BC9E467047F8B500BF3A
:08AB3000F8BC08BC9E4670470A
:10AB38002F000000434F4D4D414E442E54585400B1
:10AB480046494C45312E5458540000004552525243
:10AB58004F52212121202A25732A20646F657320F2
:10AB68006E6F74206578697374730A0A00000000B8
:10AB78004552524F52212121204E6F2E202564200C
:10AB8800696E206F70656E696E672066696C6520F6
:10AB98002A25732A0A0A00004552524F52212121C0
:10ABA800204E6F2E20256420696E207265616469CD
:10ABB8006E672066696C65202A25732A0A0A0000D8
:10ABC8004552524F52212121204E6F2E20256420BC
:10ABD800696E20636C6F73696E672066696C6520A7
:10ABE8002A25732A0A0A000046696C65202A2573FB
:10ABF8002A20434C4F534544207375636365737330
:10AC080066756C6C790A00004552524F5221212119
:10AC18002043616E2774207365656B207468652016
:10AC280066696C653A2020202A25732A0A0A0000E2
:10AC38004552524F52212121202A25732A20646F20
:10AC48006573206E6F74206578697374730A0A00DF
:10AC58002A25732A20686173206265656E207265F3
:10AC68006D6F766564207375636365737366756C61
:10AC78006C790A004552524F52204E6F2E2025649F
:10AC880020696E2072656D6F76696E67202A25735C
:10AC98002A0A0A00222A2B2C3A3B3C3D3E3F5B5DA8
:10ACA8007C7F0000232D302B20000000686C4C00B6
:10ACB80065666745464700003031323334353637EC
:10ACC80038394142434445460000000030313233B0
:10ACD80034353637383961626364656600000000D0
:10ACE800BD3C0008E53C0008ED3C0008113D0008AB
:10ACF800353D0008000000000102030400000000C8
:10AD080000000000010203040607080943554541F5
:10AD18004141414345454549494941414592924F41
:10AD28004F4F5555594F554F9C4F9E9F41494F5531
:10AD3800A5A5A6A7A8A9AAABACADAEAFB0B1B2B352
:10AD4800B4414141B8B9BABBBCBDBEBFC0C1C2C3A2
:10AD5800C4C54141C8C9CACBCCCDCECFD1D1454558
:10AD68004549494949D9DADBDCDD49DF4FE14F4F35
:10AD78004F4FE6E8E85555555959EEEFF0F1F2F323
:0CAD8800F4F5F6F7F8F9FAFBFCFDFEFF0D
:08AD94007C5DFF7F010000005F
:04AD9C006902000840
:04ADA0004102000864
:10ADA400040000200000000080000020E8000020D3
:10ADB400500100200000000000000000000000001E
:10ADC400000000000000000000000000000000007F
:10ADD400000000000000000000000000000000006F
:10ADE400000000000000000000000000000000005F
:0CADF40001010000100000000024F40029
:040000050800AACD78
:00000001FF
